:100000000020001015010000D1000000D500000004
:1000100000000000000000000000000000000000E0
:10002000000000000000000000000000D9000000F7
:100030000000000000000000DD0000004938000062
:10004000E5000000E5000000E5000000E50000001C
:10005000E5000000E5000000E5000000E50000000C
:10006000E5000000E5000000E5000000E5000000FC
:100070000D280000E5000000955F00008D65000080
:100080004D660000E5000000496A0000C96A0000F2
:10009000E5000000E5000000E5000000E5000000CC
:1000A00000000000E5000000E5000000E5000000A1
:1000B00000000000E500000025630000C48C000083
:1000C00000000010900400009004001004190000CB
:1000D000FEE7C046FEE7C046FEE7C046FEE7C04674
:1000E000FEE7C046FEE7C04610B5002304E0046802
:1000F0000C600433043004319342F8D310BDC04681
:100100000023002202E00260043304308B42FAD361
:100110007047C04638B5164B00221A60AA229A6072
:1001200055229A60134B144C07E0186859681D1C3F
:100130000C359A68FFF7D8FF2B1CA342F5D307E0D4
:1001400018681D1C08355968FFF7DAFF2B1C00E002
:100150000A4CA342F4D30A4B1B680A4A196811607F
:100160005A68094B1A6007F0DBF807F081FAFEE7DE
:1001700000400040BC000000C8000000D0000000AB
:100180000000FC1F7C09001078090010FFFFFFFF32
:10019000FFFFFFFFFFFFFFFFFFFFFFFFFFFFFFFF6F
:1001A000FFFFFFFFFFFFFFFFFFFFFFFFFFFFFFFF5F
:1001B000FFFFFFFFFFFFFFFFFFFFFFFFFFFFFFFF4F
:1001C000FFFFFFFFFFFFFFFFFFFFFFFFFFFFFFFF3F
:1001D000FFFFFFFFFFFFFFFFFFFFFFFFFFFFFFFF2F
:1001E000FFFFFFFFFFFFFFFFFFFFFFFFFFFFFFFF1F
:1001F000FFFFFFFFFFFFFFFFFFFFFFFFFFFFFFFF0F
:10020000FFFFFFFFFFFFFFFFFFFFFFFFFFFFFFFFFE
:10021000FFFFFFFFFFFFFFFFFFFFFFFFFFFFFFFFEE
:10022000FFFFFFFFFFFFFFFFFFFFFFFFFFFFFFFFDE
:10023000FFFFFFFFFFFFFFFFFFFFFFFFFFFFFFFFCE
:10024000FFFFFFFFFFFFFFFFFFFFFFFFFFFFFFFFBE
:10025000FFFFFFFFFFFFFFFFFFFFFFFFFFFFFFFFAE
:10026000FFFFFFFFFFFFFFFFFFFFFFFFFFFFFFFF9E
:10027000FFFFFFFFFFFFFFFFFFFFFFFFFFFFFFFF8E
:10028000FFFFFFFFFFFFFFFFFFFFFFFFFFFFFFFF7E
:10029000FFFFFFFFFFFFFFFFFFFFFFFFFFFFFFFF6E
:1002A000FFFFFFFFFFFFFFFFFFFFFFFFFFFFFFFF5E
:1002B000FFFFFFFFFFFFFFFFFFFFFFFFFFFFFFFF4E
:1002C000FFFFFFFFFFFFFFFFFFFFFFFFFFFFFFFF3E
:1002D000FFFFFFFFFFFFFFFFFFFFFFFFFFFFFFFF2E
:1002E000FFFFFFFFFFFFFFFFFFFFFFFFFFFFFFFF1E
:1002F000FFFFFFFFFFFFFFFFFFFFFFFFFFFFFFFF0E
:10030000054AD023D0588021C9000143D150D1588B
:1003100010208143D15070470040044008B50120AF
:100320000521012201F000FF01200521002201F03A
:100330003BFFFA20400006F087F80120052101224A
:1003400001F032FF01200521002201F0EDFE1E2008
:1003500006F07AF80120052101F05EFF08BDC046D5
:1003600070B5061C01200521012201F0DDFE0120EF
:100370000521012201F018FF0025012424E0201CA2
:100380000521002201F010FF231C33400BD0062072
:1003900006F05AF8201C0521221C01F005FF502010
:1003A00006F052F80AE0502006F04EF8201C052115
:1003B000221C01F0F9FE062006F046F87608201C03
:1003C00006F042F80135EDB2072DD8D901200521FC
:1003D000002201F0A9FE70BDF8B55F4656464D46B5
:1003E0004446F0B483468A46002291460027012401
:1003F00037E0D846C844424617703D1C261C2AE008
:10040000201C0521221C01F08FFE201C05213A1C16
:1004100001F0CAFE201C06F017F8201C0521221C42
:1004200001F0C2FE201C05213A1C01F07DFE0220D5
:1004300006F00AF8201C052101F0EEFE002803D08A
:1004400042461378334313702A2005F0FDFF7600EF
:10045000F6B20135EDB2072DD2D94B460133DBB2EE
:100460009946D145C5D33CBC90469946A246AB4679
:10047000F8BDC04638B5011C164B8E229200985824
:100480001024A043985080229C588020C001204313
:1004900098500023104D002402E09A00545101337B
:1004A000072BFAD90D4AB423D0588724A043D05043
:1004B000D45803202043D050094B186807F009FD99
:1004C0000138FF220240120201231A43054B1A6031
:1004D00038BDC04600800440800900100040044040
:1004E00088040010000002400023072282425B4182
:1004F0005B4218400E4B1A68FF218A431A60196844
:10050000012282400A43802149040A431A60094BB0
:10051000C21892001368002BFCDA054A10680649DD
:100520000140116000205A0001D41B04980D70474F
:100530000000024004800010FFFFFFF808B5012012
:100540000121012201F0F0FD0121C023014AD15017
:1005500008BDC0460040044008B5002807D000236D
:10056000074A1360074A1370074A137006E02F23E7
:10057000064AD25C0120012101F016FE08BDC046EA
:10058000980400109404001096040010E80F001066
:1005900008B5614A136801331360604A926B934255
:1005A00007D92F235D4AD35C9A0702D501225C4B01
:1005B0001A702E23594AD35C002B00D1AAE0594B64
:1005C0001B68012B20D0002B05D0022B62D0032BFF
:1005D00000D185E09EE02F23504AD35CDA0705D591
:1005E00001200121012201F0DFFD04E001200121B1
:1005F000002201F0D9FD484B1B68052B00D889E08B
:100600000122484B1A6085E0444B1B6B834203DB9D
:10061000434B1B78002B39D0434A13780133DBB2AC
:100620001370032B03D83E4B1B78002B72D02F2363
:100630003A4AD35CDA0705D501200121002201F0F6
:10064000B3FD04E001200121012201F0ADFD2F23C3
:10065000324AD35C9A0708D50322324B1A603423FE
:100660002E4AD25C314B1A7054E000222E4B1A7085
:100670002A4B9A6B284B1B689A4203D20522294BBE
:100680001A6047E00222274B1A6043E00022264B03
:100690001A703FE0214B1B6B83421DDD224A137809
:1006A0000133DBB21370032B34D92F231B4AD35CE5
:1006B000DA0705D501200121012201F075FD04E0D2
:1006C00001200121002201F06FFD0022164B1A705B
:1006D0000122144B1A601DE00022134B1A7019E01E
:1006E000124A1378013BDBB21370002B12D10522A2
:1006F0000C4B1A602F23094AD35CDA0705D5012079
:100700000121012201F050FD04E00120012100221D
:1007100001F04AFD08BDC04690040010E80F00102B
:100720009504001098040010960400109404001022
:1007300008B5002802D0012805D009E000200C21CE
:1007400001F06AFD05E00220002101F065FD00E0F6
:10075000002043425841C0B208BDC0461D4B002294
:100760001A70E121490259605A701A7201215972B6
:100770003C20D8601A611975174898611748D861EC
:1007800020201A5421201A5459842421012058541D
:100790009621890199622C215A54114B1B78012B07
:1007A00003D902212C230B4AD1540A4B11212D22AB
:1007B000995400222E215A542F215A540949196361
:1007C000032034215854044999633C215A543D2153
:1007D0005A547047E80F001050460000A0800200F5
:1007E00004000010A086010008B5FFF7B7FF08BDA0
:1007F00004E00A7802701A1C01310130531E002AED
:10080000F7D17047C9B202E001701A1C0130531EC3
:10081000002AF9D17047C04670B5031C002001E0E2
:10082000291C331C541E002A07D05E1C18784D1C4E
:100830000B78C01A221C0028F2D070BD00E00130F5
:100840000378002B01D08B42F9D1181C7047C046A9
:10085000F8B55F4656464D464446F0B489460C68A6
:1008600000E0013423782F2BFBD05C2BF9D0866974
:10087000301C20210B22FFF7C5FF23782E2B1DD122
:10088000002100235A1CE35C2E2B05D1022A03D839
:100890007354131C0131F5E72F2B05D05C2B03D0CB
:1008A0000620202B00D99DE0A21849460A6020228C
:1008B000202B00D82422F272002093E0002700238E
:1008C000082290469B465A1C9246E55C202D58D93A
:1008D0002F2D56D05C2D54D02E2D01D047450DD351
:1008E0004346082B75D12E2D75D159468B00DBB2AE
:1008F0009B46534608270B229046E4E76BB2002B39
:1009000003DA0323594619438B462B1C7F33DBB292
:100910001E2B04D92B1C2033DBB21C2B14D85346BE
:1009200001335146625C111C40393E2903D94039DC
:10093000C9B27C2951D841460139B9424FD9791CF5
:10094000F55502377254BEE72948291CFFF776FF98
:10095000002846D12B1C413B192B04D802235A46B0
:100960001A43934609E02B1C613B192B05D8012340
:10097000594619438B46203DEDB2F5550137534694
:10098000A1E754444A46146000232022AA425B4156
:100990009B000620002F25D03278E52A01D10522C0
:1009A00032704146082903D159468A00D2B2934693
:1009B000032259460A40012A01D1102213430C2276
:1009C00059460A40042A01D108221343F372002039
:1009D00008E0062006E0062004E0062002E00620EB
:1009E00000E006203CBC90469946A246AB46F8BDC6
:1009F00050800000F0B5474680B4041C0E1C056B07
:100A00008D4233D00379002B1FD03421091888463A
:100A100040782A1C012304F027FA031C0120002B34
:100A200025D12371626A216A5318AB420DD9E77848
:100A300009E0226AAD18607841462A1C012304F0BF
:100A400013FA013FFFB2012FF3D80020002E0ED081
:100A5000211C34316078321C012304F0BFF9031CDF
:100A60000120002B03D12663002000E0002004BCFD
:100A70009046F0BD10B5041C0A1C011C34314078AE
:100A8000012304F0ABF90323002833D11A4BE15CB6
:100A900009021A4BE35C194309B20223184A914236
:100AA00028D16D23E25C12066C23E35C1B041A431D
:100AB0006B23E35C1B021A436A23E35C1A431202B2
:100AC000120A104B9A4214D08923E25C1206882342
:100AD000E35C1B0413438722A25C120213438622A9
:100AE000A25C13431B021B0A074A9B185A1E934120
:100AF00000E00023181C10BD330200003202000089
:100B000055AAFFFF46415400BABEABFF08B5031E0D
:100B10000DD002780920002A0CD0DA888A4209D147
:100B2000587804F09BF8C30703D5032002E009209E
:100B300000E0002008BDC046F8B55F4656464D4669
:100B40004446F0B4161C03681C78303C092C05D8C8
:100B50005A783A2A02D10233036001E0C44B1C7870
:100B60000B20002C00D07CE1A300C24A9D580D60F0
:100B7000002D00D172E12B78002B0ED0687804F0A4
:100B80006DF8031CD80708D40020002E00D168E1BE
:100B90005B070A20DB17184063E100232B70E0B2EB
:100BA000687004F085F8031C0320D90700D558E1CC
:100BB000002E03D00A205A0700D552E1281C00213C
:100BC000FFF758FF031C002401281BD1FB22520011
:100BD000AA5C002A16D0FE23FF33EC5C2406FE2319
:100BE0005B00EB5C1B041C43FC23FF33EB5C1B0230
:100BF0001C43FD235B00EB5C1C43281C211CFFF7FE
:100C000039FF031C032B00D12AE10D20002B00D05B
:100C100027E14023EA5C12023F23EB5C1A4312B245
:100C200080239B009A4200D01BE14B23EF5C3F02E4
:100C30004A23EB5C1F430DD15B23EF5C3F065A2335
:100C4000EB5C1B041F435923EB5C1B021F4358231F
:100C5000EB5C1F432F624423EB5CEB705A1E0D20AC
:100C6000012A00D9FDE07B439B464123E95CA97042
:100C7000002900D1F5E04B1E0B4200D0F1E04623E5
:100C8000EA5C12024523EB5C1A4390462A81120764
:100C900000D0E6E04823EA5C12024723EB5C1343F2
:100CA0000DD15723EA5C12065623EB5C1B041A4352
:100CB0005523EB5C1B021A435423EB5C1343432282
:100CC000A85C00024222AA5C104381460D204E46D9
:100CD000002E00D1C5E0321C5A4446463009121895
:100CE00092460D20934200D2BBE0981A07F0F1F82B
:100CF000031C0D20002B00D1B3E05F4E9E42B64195
:100D0000764201365D4A934200D903260233EB61F5
:100D100050462218EA62494662186A62032E15D1CB
:100D20000D204246002A00D09BE06322A95C090600
:100D30006222AA5C120411436122AA5C12021143CE
:100D40006022AA5C0A43AA629B0010E00D20414683
:100D5000002900D185E05A44AA62022E01D15B002D
:100D600005E003225A43520801210B40D318444A9C
:100D70009B185B0A0D209F4273D301235B422B61BA
:100D80000023EB60032E5DD16B716523EA5C1202D8
:100D90006423EB5C1A4312196A61291C34316878A8
:100DA000012304F01BF800284CD1364BEA5C1202F8
:100DB000354BEB5C1A4312B2344B9A4242D1372383
:100DC000EA5C12063623EB5C1B041A433523EB5C0A
:100DD0001B021A433423EB5C1A432D4B9A4231D148
:100DE0002C4BEA5C12062C4BEB5C1B041A432B4B7E
:100DF000EB5C1B021A4386239B00EB5C1A43284BD7
:100E00009A421FD1274BEA5C1206274BEB5C1B046E
:100E10001A43264BEB5C1B021A4388239B00EB5CB6
:100E20001343EB60224BEA5C1206224BEB5C1B0483
:100E30001A43214BEB5C1B021A4387239B00EB5C9C
:100E400013432B612E701D4A138801339BB213800C
:100E5000EB80002028632871A86102E00C2000E0EC
:100E600001203CBC90469946A246AB46F8BDC04620
:100E70009C040010A0040010F50F0000F5FF000016
:100E8000FF010000330200003202000055AAFFFFFC
:100E9000525261411B0200001A02000019020000B8
:100EA0007272416123020000220200002102000050
:100EB0001F0200001E0200001D0200009E04001020
:100EC000F8B5041C0021FFF795FD051E53D12378CA
:100ED000032B48D16379002B45D000262663271CBD
:100EE0003437381C002180229200FFF78BFC5522FA
:100EF000224BE254AA22224BE25452233422A3541E
:100F00003522A35461233622A3544122372162544F
:100F100072218620800021541A4821541A496254B3
:100F20001A4AA354236987229200A354190A184A23
:100F3000A154190C174AA1541B0E174AA354E36875
:100F400088229200A354190A144AA154190C144A75
:100F5000A1541B0E134AA3546078391C6269012303
:100F600003F082FF667160780021002203F0CCFF5D
:100F7000002800D00125281CF8BDC0463202000020
:100F800033020000190200001A0200001B020000D8
:100F90001D0200001E0200001F02000021020000CE
:100FA0002202000023020000031C0239C269023A37
:100FB00000208A4203D998784843DB6AC0187047FA
:100FC000F8B5051C0C1E012C61D90120EB698B4280
:100FD0006DD92B78022B28D0032B3BD0012B58D175
:100FE0004E088E19710A6B6A5918281CFFF702FD0A
:100FF000002851D1F305DB0DEB1830331F79013692
:10100000710A6B6A5918281CFFF7F4FC002846D1B6
:10101000F605F60DAD193035287900020743380979
:10102000E30744D43805000D41E0090A6B6A5918FA
:10103000281CFFF7DFFC002834D16400FF235B008D
:101040001C402B193433587800022C193034237982
:1010500018432CE0C9096B6A5918281CFFF7CAFC11
:10106000002822D1A400FE235B001C402B1934333E
:10107000D87800069A78120410435B781B02184354
:101080002C19303423791843000100090FE00120A6
:101090000DE0012040420AE00120404207E001202B
:1010A000404204E00120404201E001204042F8BDFE
:1010B00070B5041C0D1CE1808168022001293DD01F
:1010C0002368DA698A4239D9002903D11A78032AB8
:1010D00000D1996A002909D1E1601A890220AA4247
:1010E0002CD99A6A2B09D318236119E09E7836010E
:1010F0000DE02068FFF764FF011C431C19D0012894
:1011000019D92368DB69834217D9AD1BADB2B5424B
:10111000EFD2E1602068FFF747FF2B09C01820617C
:101120000F231D406B012268D31834336361002004
:1011300004E0012002E0022000E0022070BDC04671
:10114000F8B5051C0C1C161C0220012979D9EB6985
:101150008B4276D92B78022B41D0032B53D002201F
:10116000012B6CD14F08CF19790A6B6A5918281CCA
:10117000FFF740FC002862D1FB05DB0D0122144083
:101180000AD0EA1830321079FF21314009010F22CC
:1011900002400A43D2B200E0F2B2EB1830331A71C7
:1011A000013701232B71790A6B6A5918281CFFF744
:1011B00021FC002843D1FF05FF0D002C02D0360989
:1011C000F6B208E0EA19303211790F229143360560
:1011D000320F0E1C1643EF1930373E712FE0090A0B
:1011E0006B6A5918281CFFF705FC002827D16400FA
:1011F000FF22520014402A1934322C19303426713F
:10120000360A56701BE0C9096B6A5918281CFFF78B
:10121000F1FB002813D1A400FE22520014402A1929
:101220003432D1782C193034090909070E4326715C
:10123000310A5170310C9170360ED670FFE70122E1
:101240002A71F8BDF0B5474680B4051C88460029D0
:1012500006D1C668002E0ED0C269B2420DD90DE08B
:101260004146FFF7ADFE031E012B3FD9EA69464612
:101270009A4203D93FE0012600E00126341C0227F0
:101280000134EB69A34202D8012E31D93C1C281C41
:10129000211CFFF795FE002806D0421C2BD0012808
:1012A00029D0B442ECD125E0281C211C134AFFF7B9
:1012B00047FF002807D14346002B04D0281C414695
:1012C000221CFFF73DFF002808D1EC602B695A1C57
:1012D0000AD0013B2B6101236B7105E0441E604283
:1012E0004441644201231C43201C04E0012002E02D
:1012F000002000E0002004BC9046F0BDFFFFFF0F7F
:10130000F0B557464E464546E0B4041C0E1CC58851
:101310000135ADB20420002D75D02369002B72D0A9
:101320000F272F4064D101332361E168002904D1E4
:1013300022681389AB4266D95AE02B09206882786B
:10134000013A1A4254D1FFF73BFE80460220434641
:10135000012B58D9013353D02368DA69424540D86C
:101360000420002E4FD0181CE168FFF76BFF804669
:1013700007204346002B46D00220012B43D00120FA
:10138000013340D020680021FFF734FB031C01200B
:10139000002B38D120683430002180229200FFF7E2
:1013A00031FA2668301C4146FFF7FEFD3063002607
:1013B00001229246B1460DE052461A712068494614
:1013C000FFF718FB00281DD123681A6B01321A633E
:1013D0000136F6B223689A78B242EDD81A6B961BA2
:1013E0001E634346E36020684146FFF7DDFD206150
:1013F000E5807F012268D71934376761002002E059
:10140000012000E001201CBC90469946A246F0BD98
:1014100070B5041C0021FFF74BFE031C002B1CD1F0
:10142000082620682169FFF7E5FA051E14D16069D6
:101430000378002B0FD0C37A1E4205D1A1690B227D
:10144000FFF7EAF9002807D0201C0021FFF758FF1A
:10145000051EE6D000E00425281C70BDF0B583B061
:10146000041C01910B782F2B01D05C2B04D101318E
:1014700001910023A36002E003689B6983600199E6
:101480000B781F2B07D8201C0021FFF711FE051C2D
:101490000023636135E004261027201C01A9FFF713
:1014A000D7F9051E2DD1201CFFF7B2FFA169CA7A1A
:1014B00000280ED004281FD1910605D50023A36073
:1014C00063611642E9D01CE00525510719D5051CBA
:1014D00017E0164212D16369DA7A174210D05A7DAA
:1014E0001202197D0A431204D87E0002997E031C61
:1014F0000B431343A360D0E7051C02E0051C00E08A
:101500000525281C03B0F0BD70B5051C0021FFF7B0
:10151000CFFD041E11D128682969FFF76BFA041E5C
:101520000BD16A691378E52B07D0002B05D0281C56
:101530000121FFF7E5FE041EEDD0002C13D1286831
:101540002969FFF757FA041E0DD16E69301C00217E
:101550002022FFF757F9301CA9690B22FFF748F941
:101560002B6801221A71201C70BDC046F0B5474699
:1015700080B4041C0D1C0227012926D9C2698A42A5
:1015800023D900270123984618E0201C291CFFF7C7
:1015900017FD061E19D0012814D0421C14D0201C9F
:1015A000291C0022FFF7CCFD071E0ED123695A1C0F
:1015B00003D00133236143466371351CE269AA42BB
:1015C000E3D802E0022700E00127381C04BC904663
:1015D000F0BDC0460B2300280ED18300074A9B585C
:1015E000002B01D000221A70002901D000230B70BB
:1015F0008000024BC1500023181C7047A00400104B
:10160000F0B54F464646C0B48DB0061C0191171C7C
:10161000002303601F23134098461E223A4001A86E
:1016200005A9FFF789FA051C02AB0B93002804D12A
:1016300005A80199FFF712FF051C0A9C002D02D195
:10164000002C00D106251C233B424DD0002D0BD091
:10165000042D03D105A8FFF757FF051C08234246B8
:101660001A4390460A9C09E0E37A11221A4202D1F9
:101670007B0702D402E0072500E00825002D40D1B9
:10168000424612073DD502F017F9A073030AE3732F
:10169000030C2374000E60740023E37223776377D6
:1016A000A377E377627D1202217D0A431204E77E6D
:1016B0003F02A17E0F431743A376E376237563753C
:1016C000059801230371002F1BD0036B9946391C29
:1016D000FFF74CFF051E14D10598013FC76049462E
:1016E000FFF788F9051C0CE0002D0AD1E37ADA0631
:1016F00004D4BA0705D5DA0702D402E0042500E0D5
:101700000725002D0AD143461B0703D52023424657
:101710001A439046059B1B6BF3613462002D1ED16A
:101720004346B371627D1202217D0A431204E37EB7
:101730001B02A17E0B4313433361E27F1206A37F9A
:101740001B041343627F12021343227F1343F3608F
:101750000023B360B361059B3360DB88B380281C32
:101760000DB00CBC90469946F0BDC046F0B55F4642
:1017700056464D464446F0B483B0041C0F1C9046B8
:101780001E1C0023336081880068FFF7BFF9031E29
:1017900000D0C8E0A27951B20223002900DAC2E0E9
:1017A0000723D10700D4BEE0E268A368D51AA84594
:1017B00000D9B1E04546AFE0A368DA0500D08FE07C
:1017C0005A0A206881780139C9B20A40904619D175
:1017D000002B01D1206902E06169FFF7F1FB0128CC
:1017E00006D8A27980235B421343A37102239AE0B7
:1017F000411C06D1A27980235B421343A3710123CC
:1018000091E0606122689246101C6169FFF7CCFB91
:10181000002806D1A27980235B421343A3710223DF
:1018200081E08346C344690A89462DD042464A4432
:1018300051468B789A4202D942469A1A91465346AB
:1018400058784946CBB2391C5A4603F0C7FA0028EB
:1018500006D0A27980235B421343A371012362E087
:10186000A37940221A420BD0A1695A468B1A4B45E4
:1018700006D25B02F818019980229200FEF7B8FFA9
:101880004B465B0299463BE0A2695A4526D0A379B4
:101890004021194212D0534658780199012303F090
:1018A000E3FA002806D0A27980235B421343A37198
:1018B000012338E0A37940218B43A371226850783B
:1018C00001995A46012303F089FA002806D0A2792B
:1018D00080235B421343A371012324E05B46A36191
:1018E000A268D105C90D80239B005B1A9946AB42C3
:1018F00000D9A94661182431381C4A46FEF778FF02
:101900004F44A1680B1C4B44A3603268131C4B442A
:1019100033604B46ED1A02E0211C24310191002D69
:1019200000D049E70023181C03B03CBC9046994600
:10193000A246AB46F0BDC046F8B55F4656464D469A
:101940004446F0B4041C0F1C151C1E1C00233360FD
:1019500081880068FFF7DAF8031E00D0E4E0A2797E
:1019600051B20223002900DADEE00723910700D4F8
:10197000DAE0E36859190022994252415242154077
:10198000C5E0A368DA0500D0A2E05A0A2068817891
:101990000139C9B20A40904624D1002B08D12369ED
:1019A000002B09D10021FFF74DFC031C206103E04F
:1019B0006169FFF747FC031C002B00D1AAE0012B53
:1019C00006D1A27980235B421343A3710223ABE0CB
:1019D0005A1C06D1A27980235B421343A3710123D1
:1019E000A2E06361A3794021194214D0211C243163
:1019F00022685078A269012303F036FA002806D045
:101A0000A27980235B421343A37101238CE0A37965
:101A100040218B43A37122689246101C6169FFF735
:101A2000C3FA002806D1A27980235B421343A37135
:101A3000022379E08346C344690A89462ED0424690
:101A40004A4451468B789A4202D942469A1A9146A4
:101A5000534658784946CBB2391C5A4603F004FA2B
:101A6000002806D0A27980235B421343A37101238F
:101A70005AE0A2695946531A4B450BD2201C243018
:101A80005B02F91880229200FEF7B2FEA379402291
:101A90009343A3714B465B0299462DE0A1695945DA
:101AA00014D0A268E3689A4210D2211C2431524615
:101AB00050785A46012303F091F9002806D0A27904
:101AC00080235B421343A37101232DE05B46A36196
:101AD000A168C805C00D80229200121A9146AA4240
:101AE00000D9A94620182430391C4A46FEF780FE4A
:101AF000A37940210B43A3714F44A268131C4B44AC
:101B0000A36031680B1C4B4433604A46AD1A002D6C
:101B100000D036E7A368E1688B4200D9E360A27980
:101B200020231343A3710023181C3CBC9046994604
:101B3000A246AB46F8BDC04638B5041C8188006893
:101B4000FEF7E4FF002845D1A3799A0642D55A064C
:101B50000FD5211C243123685878A269012303F092
:101B600083F9031C0120002B34D1A3794022934335
:101B7000A3712068E169FEF73DFF00282AD1256A9C
:101B8000EA7A20231343EB72237B2B77A3891B0A6A
:101B90006B77A37BAB77E37BEB77237CAB76238AF6
:101BA0001B0AEB76A37C2B75638A1B0A6B7501F00D
:101BB00083FEA875030AEB75030C2B76000E68767E
:101BC000A37920229343A371012322681371206813
:101BD000FFF776F938BDC04610B5041CFFF7ACFF1F
:101BE000002801D10023236010BDC046F0B5574640
:101BF0004E464546E0B4041C0D1C81880068FEF783
:101C000085FF061C002E00D0CBE0A3795AB202203B
:101C1000002A00DAC5E0E268AA4202D2990700D49D
:101C2000151CA26890460023A360002D7DD0236878
:101C300099469F787F02002A14D0681E391C06F04E
:101C400048F9824601235B4298444046391C06F01D
:101C500040F9824506D37B4241460B40A360ED1A12
:101C600061691AE02169002916D14846FFF7EAFAAE
:101C7000011E012906D1A27980235B421343A3717F
:101C800002208EE0421C06D1A27980235B421343DE
:101C9000A371012085E02061616100292BD100251D
:101CA00046E0A2794346134205D02068FFF7CAFAFE
:101CB000011E04D124E02068FFF782F9011C4A1CB0
:101CC00006D1A27980235B421343A371012068E00F
:101CD000012903D92268D2698A4206D8A2798023D1
:101CE0005B421343A37102205BE06161A368DA19D0
:101CF000A260ED1B01E002229046BD42D1D800E077
:101D00003D1CA3685A19A260EA0510D02068FFF7AD
:101D10004BF9002806D1A27980235B421343A371BB
:101D200002203EE06D0A2D1802E0002500E00025AB
:101D3000A168CB052BD0A269AA4228D0A379590665
:101D400013D5211C243123685878012303F08CF823
:101D5000002806D0A27980235B421343A37101209F
:101D60001FE0A37940229343A371211C24312268F0
:101D700050782A1C012303F031F8002806D0A279FC
:101D800080235B421343A37101200AE0A561A3688D
:101D9000E1688B4204D9E360A27920231343A37145
:101DA000301C1CBC90469946A246F0BDF0B5574683
:101DB0004E464546E0B482B082469146051C00245A
:101DC0000139884601AE0FE04846311C01226B46BE
:101DD000FFF7CCFC009B012B0AD133786F1C2B70D2
:101DE00001340A2B03D03D1CA045EDDC00E03D1C76
:101DF00000232B70631E9C4160425346184002B082
:101E00001CBC90469946A246F0BDC04600B583B0C2
:101E10006B461870081C6946012201ABFFF78CFD68
:101E200001980138431E984140420123184303B0F2
:101E300000BDC04670B5041C0E1C002506E0311C18
:101E4000FFF7E4FF431C05D001340135207800285A
:101E5000F5D1281C70BDC0460EB4F0B55F4656469D
:101E60004D464446F0B488B0834611AB02CB07938D
:101E70000022904600270E1C3FE1741C3078002899
:101E800000D13EE125280AD05946FFF7BFFF804622
:101E9000031C013301D001218846261C2CE1B31C10
:101EA00072789146302A05D1F31CB678B1460121EB
:101EB000019109E00022019249462D2904D1F31C29
:101EC000B678B146022201921E1C00254B4607E05F
:101ED000AA0055196D00EB181D1C303D33780136F2
:101EE0001A1C303A092AF3D999466C2B01D04C2B95
:101EF00006D10423019919430191327891460136A4
:101F00004B46002B00D1FCE04A46613A192A01D821
:101F1000203BDBB21A1C423AD1B2162952D88A00B1
:101F20007F498A589746079B1A1D07921A68002412
:101F300000E00134135D002BFBD19146019B9B0710
:101F400009D50021884615E020205946FFF75EFF9D
:101F500036182C1C04E00022B246161CB8462F1C72
:101F6000651CBC42F0D35346AA463D1C4746B046CA
:101F70001E1C544648465946FFF75CFF8044B14654
:101F80004646B8462F1C05E020205946FFF73EFF85
:101F900036182C1C651CBC42F6D34746B0464E464C
:101FA000431C00D0A8E08046A6E0079B1A1D0792BC
:101FB00018785946FFF72AFF80469DE00A240AE078
:101FC000102408E048465946FFF720FF804693E07A
:101FD000022400E008240421019A114204D0079A47
:101FE000111D079117680AE0442B04D1079A111DAF
:101FF0000791176803E0079A111D07911768442B92
:1020000006D1002F04DA7F42082301991943019178
:102010000022A846151CB246261C00E01D1C381CD8
:10202000311C05F056FFCCB2381C311C05F051FFB5
:10203000071C092C06D907234946782900D12723F4
:102040001C19E4B26B1C303403AA5455002F01D084
:102050000F2BE3D91C1C45465646019A120703D59F
:102060002D2203AB1A550134202398460199C90744
:1020700001D5302290460027022301991940231CE4
:10208000B1462E1C0D1CA24605E040465946FFF7FE
:10209000BDFE3F18231C002D0AD15C1CB342F4D3B3
:1020A000351CA04654464E46C146A8465D4604E04F
:1020B0005446B0465D464E469946013C03AB185D1A
:1020C000291CFFF7A3FE3F18002CF6D1AB4645466E
:1020D0004B46B0465E4605E02020311CFFF796FED9
:1020E0003F18231C5C1CAB42F6D3B34646468046E1
:1020F000021C013200D0B84647444346013300D0A9
:10210000BBE64146013100D14746381C08B03CBC13
:1021100090469946A246AB46F0BC08BC03B01847AF
:10212000F47F00007047C046012817D0002802D075
:10213000022824D033E0012A08D1A023DB051A6A43
:1021400001208840011C1143196228E0A023DB050F
:102150001A6A0120884082431A6220E0012A07D1CE
:102160000F4B1A6A01208840011C1143196216E0C6
:102170000B4B1A6A0120884082431A620FE0012A41
:1021800007D1084B1A6A01208840011C11431962CB
:1021900005E0044B1A6A0120884082431A627047A6
:1021A0000000015000000250012814D0002802D085
:1021B00002281ED02AE0002A06D001238B40191CD9
:1021C000A023DB05D96021E001238B40191CA0234B
:1021D000DB0519611AE0002A05D001238B40191C88
:1021E0000B4BD96012E001238B40191C084B19617D
:1021F0000CE0002A05D001238B40191C054BD96047
:1022000004E001238B40191C024B19617047C04642
:102210000000015000000250012808D0002802D020
:10222000022807D008E0A023DB055A6804E0064B2B
:102230005A6801E0054B5A6801238B40101C184076
:10224000431E98417047C0460000015000000250F4
:1022500030B5031C0022134C002002E0910008510D
:102260000132132AFADD00210E4C002502E0013371
:10227000081C011C1A78202AF9D0002A10D0481C0A
:1022800089000B5100E001331A78002A01D02C2A72
:10229000F9D1002A05D01D7001331428E9D100E0DE
:1022A000081C30BD480A001038B50D1C8400134BC3
:1022B000E1580C780020002C1FD0012A0ED002DC3F
:1022C000002A05D018E0022A0BD0032A0FD013E011
:1022D000081C04F05BFE286001200EE02C70012039
:1022E0000BE0081C04F018FE2860012005E0281C03
:1022F00005F064FA012000E0012038BD480A001012
:1023000010B5011C0931094C201C05F057FA201C9E
:1023100004F0A6FDC0B2032803D903380022034B02
:102320001A540122024B1A7010BDC046A0090010B9
:10233000AC04001010B52A4C0020211C0222FFF72B
:10234000B3FF211D01200222FFF7AEFF211C08313F
:1023500002200122FFF7A8FF211C0C3103200222DA
:10236000FFF7A2FF211C103104200122FFF79CFF80
:10237000211C143105200022FFF796FF211C183183
:1023800006200022FFF790FF211C1C3107200222AB
:10239000FFF78AFF211C203108200222FFF784FF6B
:1023A000211C243109200122FFF77EFF211C283146
:1023B0000A200222FFF778FF211C2C310B2001227A
:1023C000FFF772FF211C30310C200022FFF76CFF59
:1023D000211C34310D200322FFF766FF10BDC046DB
:1023E0000C0A0010024B187941384342584170479B
:1023F000980C0010F0B5474680B4424C0020211CD8
:102400000022FFF751FF211D01200122FFF74CFFA1
:10241000211C083102200222FFF746FF211C0C314B
:1024200003200122FFF740FF211C1031042002226B
:10243000FFF73AFF211C143105200122FFF734FF7A
:10244000211C183106200222FFF72EFF211C1C310F
:1024500007200222FFF728FF211C2031082000223C
:10246000FFF722FF211C243109200222FFF71CFF65
:10247000211C28310A200122FFF716FF224D236874
:102480002B60226A2A622148214905F055F8276A03
:10249000381C204905F01DFDC6B21F4B1E701F4B96
:1024A00098465E43F619301C642105F012FDC0B257
:1024B0001B4B187064277F4278438619FA23DB0090
:1024C000F618184B1E802668301C124905F001FDD5
:1024D000C0B2154B1870434658438619301C64210E
:1024E00005F0F7FCC0B2114B18704743BE19104BF2
:1024F0001E70281C211C2C2205F0C3F804BC904639
:10250000F0BDC046980C0010DC090010797700007F
:10251000948000001027000022000010F0D8FFFF78
:1025200008000010200000101C000010D004001053
:10253000C8040010014B18607047C046080A00101C
:10254000F8B5041C2C233C4AD35C012B01D901F0C3
:102550002DF82378242B04D03848394904F0ECFFB7
:1025600068E0201C04F07CFC061C0023002009E02D
:10257000711E61180A780A2A01D00D2A01D108704B
:10258000013E0133012BF3DDB01E201804F092FD53
:10259000021C033E0023012102E0655C6B40013117
:1025A000B142FADB834203D02448264904F0C4FF39
:1025B000601C254904F042FC002803D1201CFFF7D1
:1025C0009FFE37E00023A371A6193370E01DFFF7CB
:1025D0003FFE051C0334201C1C4904F02FFC00287E
:1025E00006D11B4B1B68DA0702D5281CFFF7A2FE99
:1025F000201C184904F022FC00281BD1144B1B6836
:10260000DA0617D5144B1B78022B10D108E0A30073
:10261000D85904F0DDFC301C04F0DAFC013402E08F
:1026200000240E4F0E4EAC42F1DB04F063FD281C7B
:10263000FFF7E0FEF8BDC046E80F00107977000014
:10264000A4800000C0800000FC8000000481000025
:10265000080A001008810000A4040010480A0010B5
:102660000C81000008B5034B996A012004F0D8FAE8
:1026700008BDC046E80F001038B52DE0012004F079
:10268000A1FB051C041E27D024280AD10022154BCB
:102690001A60154B1B78012B03D11448144904F020
:1026A0004BFF104A1368134AD554FF22520093423D
:1026B00002DC01330B4A13600B4A1378012B02D161
:1026C000281C00F02BFD0D2C06D1064B1B68094879
:1026D0000022C254FFF734FF012004F06DFB0028F4
:1026E000CCD138BDA8040010A404001079770000F4
:1026F00050890000980A001038B5174B1B78002B42
:1027000028D1164B1B78022B07D01548154905F028
:1027100055F80122104B1A701CE00422124B1A705B
:102720002423124AD05C12490D2204F029FB0E4CDE
:10273000094D01E0FFF7A0FF2378002B02D02B7892
:10274000002BF7D0044B1B78002B03D10448094918
:1027500005F034F8024838BDAC0400100400001045
:10276000A009001010810000E8040010E80F00101C
:10277000188100002881000008B58020FE2100F0AB
:10278000DFF90020142103F0C3FE08BD10B584B0AA
:10279000194B1B78012B2AD90023002103E001AA41
:1027A000D1540133DBB2082BF9D98020F52100F098
:1027B000C7F90020142103F0ABFE01AC8020211CDE
:1027C000032200F0DDF920780002637818430B4BF8
:1027D00018400B4B584300140A4BC0180A4B984240
:1027E00000DD181CC343DB17184080B200E0002056
:1027F00000B204B010BDC04604000010FCFF000091
:10280000D4300000A8FDFFFF102700008023DB0567
:102810005B68FF221340083B502B00D9B8E09B00B7
:102820005E4AD3589F465E4B00221A601A68511CBC
:1028300019605C4B9A5CD2B28023DB059A60282237
:102840009A610122584B1A60A6E00022574B1A6089
:10285000534A1368591C1160524AD25CD2B2802389
:10286000DB059A6028229A6102224F4B1A6093E09E
:102870004D4B1B68012B0CD1494A1368591C116040
:10288000484AD25CD2B28023DB059A600422464BD0
:102890001A6008228023DB059A617DE0404B1A68AC
:1028A000434B1B689A420DD23D4A1368591C116074
:1028B0003C4AD25CD2B28023DB059A6004223A4BB8
:1028C0001A6012E03B4B1B68002B07D020228023AC
:1028D000DB051A600322344B1A6006E00522324BF6
:1028E0001A6010228023DB051A6008228023DB0592
:1028F0009A6151E02F4B1B68012B04D104228023E5
:10290000DB059A6103E004228023DB051A600822BC
:102910008023DB059A613FE0244B1A68511C196043
:102920008021C9058868C0B2234988541A68214BA0
:102930001B689A4206D204231B4A13608022D205E8
:10294000136006E00522184B1A6004228023DB0581
:102950009A6108228023DB059A611DE0134B1A68F7
:10296000511C19608023DB059868C0B21249885455
:1029700005210D4A116010221A6008229A610BE0AD
:1029800008228023DB059A610522074B1A6003E0C9
:1029900008228023DB059A617047C046348100001D
:1029A000BC040010EC0C0010B4040010B0040010C3
:1029B0000C0D0010C40C0010C80C001010B5202223
:1029C0008023DB051A6000220A4B1A6000230949A4
:1029D00009480A4C05E00268012A07D0A34207D83B
:1029E00001330A68012AF6D9002002E0012000E044
:1029F000002010BDD80F0010B4040010FEFFFF002F
:102A00008023DB0510221A6008229A61191C10220B
:102A10000B681A42FCD101207047C04670B51C4BB0
:102A20005A6802210A435A6080229D5820242C4370
:102A30009C50184B90229C583F25AC439C509C586E
:102A40000C439C509E588024E40026439E509422C0
:102A50009E58AE439E509D582943995099580C4317
:102A60009C508023DB056C229A6132225A611A61E4
:102A7000022803D1A0228023DB05DA6080225201E4
:102A8000054B1A6040228023DB051A60012070BDCF
:102A9000008004400040044000E100E010B5002345
:102AA0000F4A13600F4A13600F4A1360FFF786FF47
:102AB000041E012C03D0FFF7A3FF00240EE0002228
:102AC0000A4B1A601A1C064905E00B68052B02D157
:102AD000FFF796FF02E01368092BF6D9201C10BD02
:102AE000B4040010B0040010BC040010D80F001093
:102AF00038B50E4B1870002301240C4D03E0C85C60
:102B00002855013301349A42F9DC094B1B78DA0766
:102B100004D508480549221C04F060FB064B1C60E4
:102B20000022064B1A60FFF7B9FF38BDEC0C00100D
:102B3000B8040010788200000C0D0010C40C0010C6
:102B400008B50A4B18705970094B1B78DA0704D581
:102B500008480649022204F041FB0222064B1A6093
:102B60000022064B1A60FFF799FF08BDEC0C00101D
:102B7000B8040010808200000C0D0010C40C00107E
:102B800038B50D1C141C012318430E4B18700E4B46
:102B90001A600E4B01221A60FFF780FF00230C4AD7
:102BA00003E0D05CE8540133DBB2A342F9D3094A15
:102BB0001278910704D5084805491A1C04F00EFB49
:102BC00038BDC046EC0C0010C40C00100C0D0010F9
:102BD000C80C0010B804001088820000F0B5474609
:102BE00080B4984606AB1E78194B18700024012556
:102BF00003E00F5D5F5501340135A242F9DC01238A
:102C00001843134B5855134B1B78D80704D512485B
:102C10000F492A1C04F0E2FA104B1D60104B1E6095
:102C20000021104B03E05A5C404642540131321EF1
:102C30008A42F8DC074B1B78D90703D506480949B7
:102C400004F0CCFAFFF72AFF04BC9046F0BDC04662
:102C5000EC0C0010B8040010988200000C0D00105D
:102C6000C40C0010C80C001008B5124B80229858F4
:102C70008021C9010143995098588021C90001431E
:102C80009950985840210143995098588021490201
:102C90000143995001229A6772B63922064B1A6095
:102CA000064B1B6883F30888054B1B6802480549DF
:102CB000984708BD00800440100D00100000FF1F61
:102CC00000000010240D0010BFF34F8F024A034B89
:102CD000DA60BFF34F8FFEE70400FA0500ED00E075
:102CE000F0B55F4656464D464446F0B485B00023E5
:102CF000002203E06946CA540133DBB20F2BF9D935
:102D000000229246304B9946304DA84629E00727CD
:102D100051467D1AEDB253460833DBB29C46012280
:102D200000234C0017E0215A0A4210D01E1C4F46C7
:102D3000FF5C291C002F00D061464746BE5D01277D
:102D4000B7403E1C6F467F5C3E436F467E54520048
:102D500092B20133DBB20F2BE5D956460136F6B2FB
:102D6000B24651460729D2D9194B70221A70C8228F
:102D70005A7080229A70174B1B78002B03D0F122D7
:102D8000134BDA7002E0F022114BDA706022104B24
:102D90001A71002305220E4C06E0511C6D46E85CBA
:102DA000A0540133DBB2CAB20F2BF6D90A4B1A601A
:102DB00000220A4B1A60FFF771FE05B03CBC90463A
:102DC0009946A246AB46F0BDC8830000B883000018
:102DD000EC0C0010490D00100C0D0010C40C00107C
:102DE000F0B54F464646C0B485B01A4B1A7800235A
:102DF000002A1BD0013A174B1A7026E01A1C6046B5
:102E0000C156002902DA4D461349CD54B95C490038
:102E1000895B50006D464153A05C002803D05200EE
:102E20004046014351530133DBB209E00A4884466E
:102E300000218946071C094E094C8022D201904688
:102E4000072BDBD96846FFF74BFF05B00CBC90465B
:102E50009946F0BD4A0D0010340D0010B8820000F4
:102E60004C0D001010B500220F4B1A7000230F49B3
:102E700002E0CA540133DBB2072BFAD90C4B7022A3
:102E80001A70C8225A7080229A70F022DA7060227A
:102E90001A710522074B1A600024074B1C60FFF7CC
:102EA000FDFD064B1C7010BD490D0010340D0010C7
:102EB000EC0C00100C0D0010C40C00104A0D00109A
:102EC000F8B50023114D20241149002203E0EC54F1
:102ED000CA540133DBB2072BF9D9002200210B4D74
:102EE0000B4E012709E02E2B02D1531EF75402E0AE
:102EF000541CAB54E2B20131C9B2072A02D8435C78
:102F0000002BF0D1FFF76CFFF8BDC046340D001068
:102F10004C0D001008B5FFF7D3FF1022014B1A70BB
:102F200008BDC0464A0D0010F0B5474680B484B0D5
:102F3000052800D9C2E08000624B1B589F465A000A
:102F4000684611520133DBB202E0002301214942FD
:102F5000072BF4D96846FFF7C3FE00205A4903F057
:102F6000D7FAABE05A00694654520133DBB202E0B3
:102F7000331C4446AC40072BF4D96846FFF7B0FE3B
:102F8000301C391C03F0C4FA0135EDB205E0002510
:102F9000002601229046FA277F000F2DE8D98DE008
:102FA0005A00684611520133DBB201E000230021D0
:102FB000072BF5D9002188460026012718E03B1C85
:102FC000A34068462A5A13432B52FFF789FE301C50
:102FD000FA21490003F09CFA0134E4B202E0341C07
:102FE000424655000F2CEAD943460133DBB29846DE
:102FF0004346072BF3D90020FA21C90003F088FAD1
:103000005CE05A00684611520133DBB201E0002354
:103010000021072BF5D9002188460026012717E05B
:103020003B1CA34068462A5A13432B52FFF758FE15
:10303000301C142103F06CFA0134E4B202E0341CB9
:10304000424655000F2CEBD943460133DBB298467C
:103050004346072BF3D90020FA21890003F058FAE0
:103060002CE05A00684611520133DBB201E0002324
:103070000021072BF5D90020002501271AE03B1C71
:10308000A340694673526846FFF72AFE281C03F0E6
:1030900099FE0134E4B202E02C1C424656000F2C8B
:1030A000EDD943460133DBB2984600E0A8464346DB
:1030B000072BF1D9512801D07128F7D104B004BCF5
:1030C0009046F0BDA08200008813000008B50020E3
:1030D00003210122FFF728F8002004210122FFF735
:1030E00023F8002005210122FFF71EF8002003210C
:1030F0000122FFF759F8002004210122FFF754F8BC
:10310000002005210122FFF74FF808BD08B5031C78
:103110000A1C0020191CFFF747F808BD04492022AB
:103120004B691A42FCD0024B186000207047C04621
:103130000080004010B50A4B1B680A4A126893428F
:1031400005DA094A12685C1C05490C60D054064B2C
:103150001A68034B1B68D31800221A7010BDC046B2
:10316000D40400104C120010E00400100CB410B590
:1031700082B004AA08CA0024074B1C60074B1960E0
:10318000074B186001920748049904F015F902B042
:1031900010BC08BC02B01847D40400104C12001038
:1031A000E004001035310000F0B5474680B486B029
:1031B000041C0E1C151C1F1C00281ADA4442A046D1
:1031C00003AC2D23237000236370201C04F0E8FA65
:1031D0004046291C04F07AFE061C4046291C04F0D7
:1031E00075FE0091381C0621221C331CFFF7BEFF20
:1031F0000EE0111C04F06AFE8046201C291C04F01D
:1032000065FE0091381C0621321C4346FFF7AEFFD5
:1032100006B004BC9046F0BD08B501F017FD01F002
:103220000BFD00280CD00022064B1A700020064926
:10323000FEF7D0F9002803D00448054904F07CF9D2
:1032400008BDC046680D00107C0D00101D31000047
:1032500008840000F0B5474680B4184CA54401F03E
:10326000EBFC002823D01648FFF72AFE01A81549D9
:103270000122FEF7C5F9002819D1134E134B9846C9
:10328000134F301C282101AAFEF790FD041E09D01F
:103290000D4D4046391C2A1C04F04EF9281C2821EB
:1032A00001F0D4FE002CECD101A8FEF795FC8A2396
:1032B0009B009D4404BC9046F0BDC046D8FDFFFF76
:1032C000208400002C840000B00F00101D3100008D
:1032D0003C84000010B582B00C4C0D4B1A880D4B8D
:1032E0001B780D4909780091201C0C49FEF7B4FDAC
:1032F0000B4B1A780B4B1B780B4909780091201C5B
:103300000A49FEF7A9FD02B010BDC046981500108D
:10331000200000100800001022000010448400006B
:103320001C000010D0040010C80400105C840000D1
:1033300010B501F081FC002834D01B481B49122233
:10334000FEF75EF9021E04D019481A4904F0F4F899
:1033500028E0154C201CE168FEF748FC201C1649AB
:10336000FEF77AFD201C1549FEF776FD201C144956
:10337000FEF772FD201C1349FEF76EFD201C12495A
:10338000FEF76AFD114B1A783032201C1049FEF707
:1033900063FDFFF79FFF201C0E49FEF75DFD201C1B
:1033A000FEF7CAFB10BDC046981500106C840000E3
:1033B0001D31000078840000A0840000DC8400003F
:1033C000F48400001485000024850000040000102F
:1033D0004085000054850000F0B585B0114B1B7886
:1033E000002B1CD101F028FC002818D00E4F0F4EE6
:1033F0000F4D3388684610213A1CFFF7B7FE281C92
:1034000069460122FEF7FCF8041E06D10848FEF7C3
:10341000E3FB064B1A8801321A80002CE9D005B074
:10342000F0BDC046D2040010648500000600001004
:103430007013001010B588B0324B1B78002B5FD191
:1034400001F0FAFB00285BD000222F4B1A702F4BA3
:103450001B8804A810212E4AFFF788FE2C232D4A32
:10346000D35C012B06D9294B1B88684610212A4AB8
:10347000FFF77CFE254B1A8801321A80274804A9E1
:103480000A22FEF7BDF8021E04D02548254904F0A3
:1034900053F818E001221B4B1A701422224B1A70A9
:1034A000FFF718FF214C201C21496A461232FEF713
:1034B000D3FC201CFEF740FB002204AB5A72684686
:1034C0001230FFF727FD2C23124AD35C012B17D9AA
:1034D000184869460A22FEF793F8021E04D01048E5
:1034E000104904F029F80BE0FFF7F4FE0F4C201C04
:1034F00011496A460232FEF7AFFC201CFEF71CFBA6
:1035000008B010BDD2040010680D001006000010B5
:1035100074850000E80F001084850000701300100F
:103520001D31000094850000D9040010981500108A
:10353000BC85000028100010E085000010B5144B79
:103540001B78002B22D00022114B1A701148FEF775
:1035500043FB2C23104AD35C012B02D90F48FEF702
:103560003BFBFFF7B7FE0E480E49FEF775FC2C2318
:10357000094AD35C012B01D9FFF7ACFE084C201C93
:103580000949FEF769FC201CFEF7D6FA10BDC046BB
:10359000D204001070130010E80F00102810001063
:1035A00098150010048600001C86000008B5021C57
:1035B000064B1B78002B08D02C230549CB5C012B34
:1035C00003D904480449FEF747FC08BDD2040010A3
:1035D000E80F0010281000106888000010B582B0B5
:1035E0001B4C201C1B4903F0A7FF201C1A4903F0A9
:1035F000A3FF201C194903F09FFF201C184903F06A
:103600009BFF184B1A783032201C174903F094FFA7
:10361000164B1A88164B1B78164909780091201C06
:10362000154903F089FF154B1A78154B1B7815497E
:1036300009780091201C144903F07EFFFFF75CF825
:10364000021C201C114903F077FF02B010BDC046D8
:103650001D310000DC840000E887000014850000B4
:1036600024850000040000104085000020000010A8
:103670000800001022000010448400001C0000100C
:10368000D0040010C804001004880000188800004E
:10369000F0B5474680B482B080460024094F0A4EF8
:1036A0000A4D09E06300DB5B42460092301C291C96
:1036B000221C03F041FF0134072CF3DD02B004BCEF
:1036C0009046F0BD001A00101D310000388800003F
:1036D00038B5084D084B1A68084C281C0849231CAB
:1036E00003F02AFF074B1A68281C0749231C03F024
:1036F00023FF38BD1D310000181A0010508900004A
:1037000044880000141A00105088000008B5031CFB
:10371000034A12680348044903F00EFF08BDC0467F
:10372000601300101D3100006488000038B5051CCE
:103730000F4C2068642104F0C9FB021C0D480E499F
:1037400003F0FAFE2068642104F0C0FB0C1E092C73
:1037500002DC3020FFF7E2FC002C02D13020FFF722
:10376000DDFC04480549221C2B1C03F0E5FE38BD96
:10377000C41700101D3100006C8800007488000020
:1037800038B5051C074B1868074C08496422231CF0
:10379000FFF70AFD06480749221C2B1C03F0CCFE4C
:1037A00038BDC046941500105C0D00107C880000E8
:1037B0001D3100008488000038B5051C074B1868CF
:1037C000074C08490A22231CFFF7EEFC064807496C
:1037D000221C2B1C03F0B0FE38BDC0465013001055
:1037E00068130010908800001D31000098880000C8
:1037F00038B5051C104C0023E05E642104F066FB24
:1038000002B20E480E4903F097FE0023E05E6421E9
:1038100004F05CFB0CB2092C02DC3020FFF77EFCCC
:10382000002C02D13020FFF779FC04480549221C06
:103830002B1C03F081FE38BD580D00101D31000017
:10384000A48800007488000008B5154B1A6801327E
:103850001A60144B1A6801321A60134A1378013344
:10386000DBB21370632B0DD900220F4B1A700F4B74
:103870001A6801321A600E4B1B78002B02D0013BF4
:103880000B4A13700B4B1B78022B07D100201D2114
:10389000FEF7C2FC011C0420FFF738FC08BDC0463F
:1038A000C0040010D80F0010DD0F0010201A001007
:1038B000E80400100400001070B50D4B1D880D4B7E
:1038C00018780D4B1C780D4B19780D4B1A780D4B51
:1038D0001B780D4EAD196D06400528432404204386
:1038E000C9020843520110435B08184370BDC0462B
:1038F0002000001008000010220000101C00001022
:10390000D0040010C804001044F8FFFF084B1B78D7
:10391000002B0BD1074B084A196811600749084A68
:1039200011600121024A117000221A607047C046DE
:10393000D1040010601300106C0D0010F1D8FFFFCF
:10394000C017001000B583B0FFF774FD284B1B783B
:10395000002B4AD02023274AD35C002B02D0012B16
:1039600004D006E06622244B1A7002E06D22224B3E
:103970001A7021231F4AD35C002B02D0012B04D0E4
:1039800006E046221D4B1A7002E043221B4B1A70C0
:103990001A4B1B78184A12780092194819491A1CB8
:1039A000FEF75AFA2C23134AD35C002B0BD02023AA
:1039B000D35C9A00D318144AD2180F4B1B781048C6
:1039C0001249FEF749FA124B1B78012B03D90C4818
:1039D0001049FEF741FA0A480F49FEF73DFA054B38
:1039E0001B7A032B01D1FFF791FF03B000BDC04646
:1039F000D2040010E80F0010700D0010DC0F001052
:103A000070130010AC8800000C000010F08800005B
:103A10000400001038890000348800000023044AA4
:103A200013600449044A1160044A13707047C04689
:103A30006C0D0010F1D8FFFFC0170010D10400106A
:103A4000F0B55F4656464D464446F0B4B3B0FFF776
:103A5000E5FFE54A8023D158E4480143D150FEF701
:103A600061FB00200021FEF7D7FB002802D10222D3
:103A7000DF4B1A70FFF72AFB02F068FCFCF75EFDD3
:103A8000DC4B0322B4215A50B8215A500221BC22E7
:103A90009950D94B1868642104F01BFAD74B98420F
:103AA00010D80202120A013AD54B5A60D54A106A60
:103AB0000002000AC02109060143116200229A6037
:103AC00007221A60FCF790FECF4B5878596803F034
:103AD000A7F8C94B1868642104F0FBF9421E0020C6
:103AE000012102F0D9FE002002F010FEC74C201C7C
:103AF000C74903F021FD0120FEF790FF201CC549B6
:103B000003F01AFDFFF7AEF90420FFF70DFAC248E3
:103B1000FFF7D6F90020C14902F0FAFCC048FFF7D0
:103B2000CFF90020FA21890002F0F2FCBD48FFF72E
:103B3000C7F9BD48FCF79EFC0023002204E0990071
:103B4000BA480A500133DBB2022BF8D9B848FFF764
:103B5000B7F9FCF7D5FBFCF7E1FBC820400002F009
:103B600073FCCC20FCF7FCFB3C2002F06DFC4420F5
:103B7000FCF7F6FB3C2002F067FC9D4B1B78022B08
:103B800001D1FEF7F9FDAB48FFF79AF9984B1B7886
:103B9000012B02D90122A84B1A70A74B1B78012BCD
:103BA00002D102F08FF901E002F060F8A348FFF7BC
:103BB0006FFD0023A24A1360A24A13700A21A24A91
:103BC0001170A24A1360A24AA24B1A60A248FFF7E2
:103BD00077F9FFF721FBA148FFF772F9FFF73AFBEE
:103BE000894B5B7A012B02D0022B05D007E0864B74
:103BF000DA689B4B1A6002E00122994B1A60824BF3
:103C00001B7D012B02D0022B05D007E07E4B9A6969
:103C1000944B1A6002E00122924B1A607A4B1B7A95
:103C2000022B02D10122904B1A609048FFF748F90D
:103C3000FEF718FD2D23744AD05CFEF77BFC8C4BFD
:103C400000229A604E2119731A61572119759A61E1
:103C5000DA61884B1A620020874902F059FCFEF7AE
:103C60000BFD8648FFF72CF9FFF762FBFFF7B4FB6B
:103C70005F4B1B78022B02D1012003F017FB0020C1
:103C8000FCF756FD041C0120FCF752FD031C012C1F
:103C900013D1012811D17A48FFF712F98023DB05EF
:103CA00080225A611A61664C261C00252368042B69
:103CB000FCD9356001F028FFF8E7012B01D101F0B4
:103CC00081F9FEF719FD021C6E4C201C6E49FEF7AF
:103CD000C3F8201CFDF730FF6C48FFF7F1F8002116
:103CE000884600221F9200231E93002022902091DC
:103CF000534A9146934666488246FEF7BDFC4946C4
:103D00000B68042B01D800F01AFD00235A461360FB
:103D1000494B1B78012B02D102F0EAF801E001F0D7
:103D2000B7FF01F0DFFF01F0FBFF5A4B18602123C2
:103D3000354AD35C002B09D1C3001818052104F0C3
:103D4000C5F8C8231B01C018524B186002F004F8D4
:103D5000514B18603D4B1968401818603A4A137867
:103D6000013BDBB21370002B00D0E8E00A22364B97
:103D70001A700A2104F0AAF8484B186002F05EF8A5
:103D8000474B18602023204AD35C012B06D15246B2
:103D90005043444904F09AF8414B1860404A424B62
:103DA0001B681068C31A13600021284A1160294A51
:103DB0001268934201DD274A13600620FCF794FB4A
:103DC00080B23A4B18803A4B58438012394B5843D3
:103DD000FA21890004F07AF8374B18600024374E36
:103DE000334F124D77E0C046008004401F0001E0D1
:103DF000040000100040044088040010FFFFFF0092
:103E000010E000E000ED00E0E80F00101D310000C0
:103E1000488900005489000060890000DC0500002A
:103E20006C89000078890000405489005413001008
:103E30008489000090890000D80400105089000097
:103E4000C0040010DD0F0010E40F0010740D00100E
:103E5000F1D8FFFFC01700109C890000A489000062
:103E6000DC040010E4040010CC040010B089000051
:103E7000DC0900100C0A001098080000BC89000042
:103E8000C889000098150010D0890000F089000052
:103E90001027000094150010640D0010C4170010C6
:103EA00060130010288000006C0D0010DE0F001061
:103EB000E40C0000D6100000BC1700101800001021
:103EC000305DFCF711FB0004000C78438012A30066
:103ED00058510134E4B2022CF2D92099002902D0C1
:103EE000012909D017E003200121FFF70FF9052070
:103EF0000021FFF70BF90EE0DB4B1B78002B03D002
:103F000003200021FFF702F905200121FFF7FEF849
:103F100001235B422093D54B1B78012B0CD1FEF77C
:103F200061FA002804D004200021FFF7EFF803E035
:103F300004200121FFF7EAF8209A0132209243463B
:103F40000B2B00D90DE19B00C94AD3589F46C94BA2
:103F50001B682FA80C21C84AFFF708F92FA8FEF705
:103F6000AFFFFEE0C54B1B682FA80C21C44AFFF72A
:103F7000FDF82FA8FEF7A4FFF3E0C24B18680A2152
:103F800003F0A4FFC04EC14C311C0A22231CFFF7D2
:103F90000BF9BF4B1868BF4D311C0A222B1CFFF7D1
:103FA00003F900952FA80C21BB4A231CFFF7DEF86C
:103FB0002FA8FEF785FFD4E0B84B1C68201C6421B5
:103FC00003F084FF051C201C642103F07FFF009197
:103FD0002FA80C21B24A2B1CFFF7C8F82FA8FEF718
:103FE0006FFFBEE0AF4B1F68381CE121090103F0F1
:103FF00070FFFF26341C0440AB4D6543ED19281CAF
:104000003C2103F066FF06403301F31A9B005D1963
:10401000009601952FA80C21A44A231CFFF7A6F8AF
:104020002FA8FEF74DFF9CE0A14B1C68201CFA2135
:10403000890003F04BFF051C201CFA21890003F0C6
:1040400045FF00912FA80C219A4A2B1CFFF78EF8F0
:104050002FA8FEF735FF84E0279804B2201C6421C6
:1040600003F034FF05B2201C642103F02FFF09B2D6
:1040700000912FA80C21904A2B1CFFF777F82FA84E
:10408000FEF71EFF6DE08D4DAC68201C514603F01D
:104090001DFF4E1D2D7B201C514603F017FF041CF5
:1040A000301C0A2103F012FF009001952FA80C216B
:1040B000834A231CFFF75AF82FA8FEF701FF50E0B0
:1040C0007E4D2C69201C514603F000FF0E1C323639
:1040D0002D7D201C514603F0F9FE041C301C642188
:1040E00003F0F4FE009001952FA80C21754A231CC3
:1040F000FFF73CF82FA8FEF7E3FE32E02398514685
:1041000003F0E4FE041C2398514603F0DFFE009107
:104110002FA80C216C4A231CFFF728F82FA8FEF7C4
:10412000CFFE1EE0654BDC69201C514603F0CEFE3D
:10413000051C201C514603F0C9FE00912FA80C213C
:10414000624A2B1CFFF712F82FA8FEF7B9FE08E011
:104150002FA80C215E4A249BFFF708F82FA8FEF732
:10416000AFFE01F0D1FC0020FCF7E2FA041C0120B4
:10417000FCF7DEFA051C031C1E998C4223D01E940A
:10418000002C20D142460132D2B29046374A1278F2
:10419000012A05D84246062A02D10132D2B29046FF
:1041A00000220B214046814252415242104080463B
:1041B0002C2248498A5C1E94002A04D1062802D980
:1041C0001E94002188461F9A93420DD01F95002B04
:1041D0000AD1254B1B78002B03D0FFF7AFF91F95B1
:1041E00002E0FFF7AFFB1F952E4B1B682298984209
:1041F00000D1A4E2374B1B7A022B0AD1364A13684E
:10420000013B1360002B04D10022324B1A72FFF7DE
:104210007DFB304B5B7A012B02D0022B10D01BE0D0
:104220002E4A1368013B1360002B15D10022294B45
:104230005A720D4B1B78002B0ED1FFF783FB0BE05E
:10424000094B1B78002B07D10A4B1A68214B1B69BD
:104250009A4201D3FFF776FB1E4B1B7D012B3FD00B
:10426000022B4DD058E0C046D204001004000010CC
:10427000D883000060130010F8890000C0170010F8
:10428000008A000094150010908800005C0D00105A
:104290005013001068130010088A0000C4170010A3
:1042A000108A0000201A0010F0F1FFFF1C8A0000A5
:1042B000BC1700102C8A0000388A0000DC090010AE
:1042C000488A0000548A0000608A00006C8A00005E
:1042D000788A0000E80F0010CC040010DC04001005
:1042E000B54A1368013B1360002B15D10022B34B74
:1042F0001A75B34B1B78002B0ED0FFF71FF90BE09C
:10430000AF4B1B78002B07D0AE4B1A68AB4BDB6969
:104310009A4201D2FFF712F93C23A84AD35C012B41
:1043200003D12498FCF734F903E0A64B1868FCF796
:104330002FF90022A44B1A70A44B1B682293FBF7A1
:10434000EDFFC820400002F07FF8CC20FCF708F811
:104350003C2002F079F8BE20FCF702F83C2002F085
:1043600073F86C46BA34201C0221FCF735F80021A2
:10437000635E9A00D3185A00D3171B0F9B181B11AA
:10438000934A136021228D498A5C002A08D1D80003
:10439000C018052103F09AFD4130FF308C4B1860A6
:1043A000FBF7BCFFC820400002F04EF8CC20FBF722
:1043B000D7FF3C2002F048F84420FBF7D1FF3C2017
:1043C00002F042F8834B1B78022B03D1FEF7DEF993
:1043D00080B22790804B186880496422804BFEF79A
:1043E000E3FE7B4B18687F490A227F4BFEF7DCFE19
:1043F0002023724AD45C002C0BD17C4B186A5146A6
:1044000003F064FD7A4B5843514603F05FFD24905E
:1044100005E0764B186A514603F058FD2490002CB5
:104420000ED1744B9869142103F050FD724B584320
:10443000514603F04BFD83001818800023900DE0D7
:104440006C4B9869142103F041FD6C4B5843514665
:1044500003F03CFD83001818800023902C23574A5A
:10446000D35C002B00D1D5E0584B1B682893644BDC
:104470001B681D93534B1B682993624B1F68624B4B
:104480001E685D689C685B4B1A682A929868219048
:10449000197B2B911A692592187D2C90DB69269344
:1044A000FDF7A0FF2D901D98642103F00FFD0090F3
:1044B0001D98642103F00AFD0191494B02934A4B78
:1044C000039329990491381CFA21890003F0FEFC1A
:1044D0000590381CFA21890003F0F8FC0691301C85
:1044E000FA21890003F0F2FC0790301CFA218900C0
:1044F00003F0ECFC0891281CFA21890003F0E6FC8B
:104500000990281CFA21890003F0E0FC0A91201C84
:10451000FA21890003F0DAFC0B90201CFA218900B3
:1045200003F0D4FC0C912A9A0D922198514603F085
:10453000CDFC0E902198514603F0C8FC0F912B9BA7
:1045400010932598514603F0C1FC119025985146CF
:1045500003F0BCFC12912C9813902398514603F061
:10456000B5FC14902398514603F0B0FC15912698A1
:10457000514603F0ABFC16902698514603F0A6FC7A
:104580001791249918912D9A1992279B1CB2201CDF
:10459000642103F09BFC00B21A90201C642103F0FC
:1045A00095FC09B21B91194880214900184A289BA3
:1045B000FEF7DCFD90E0C046E4040010E80F0010B8
:1045C000D2040010601300101C1A0010201A0010F2
:1045D0005013001004000010941500107C88000097
:1045E0005C0D001090880000681300100C0A001089
:1045F00028800000DC090010F42C0000584800005E
:10460000C4170010BC1700105413001050120010F3
:10461000808A00004B4B1B681D934B4B1F684B4B14
:104620001E685D689C684A4B1B6821931D98642135
:1046300003F04CFC00901D98642103F047FC0191AD
:10464000444B0293444B0393444B1B680493381C24
:10465000FA21890003F03AFC0590381CFA21890000
:1046600003F034FC0691301CFA21890003F02EFC83
:104670000790301CFA21890003F028FC0891281CBF
:10468000FA21890003F022FC0990281CFA218900F4
:1046900003F01CFC0A91201CFA21890003F016FC8F
:1046A0000B90201CFA21890003F010FC0C91279834
:1046B00004B2201C642103F009FC00B20D90201C00
:1046C000642103F003FC09B20E91254880214900C2
:1046D000244A219BFEF74AFD234B1B78002B04D074
:1046E000224823491E4A02F027FF224B1B78002B49
:1046F00025D0214A1388013B9BB21380002B1ED189
:104700001E4B5A8C1C4B1A801D4B1A6801321A60C2
:104710001C481D49124AFDF79FFB0D4B1B683F22A9
:10472000191C91438B420AD11648FDF705FA2C2338
:10473000124AD35C012B02D91448FDF7FDF930BFB2
:10474000FFF7DBFAC4170010BC1700105413001059
:10475000201A00105C0D0010681300106013001088
:1047600050120010008B0000D30400101D31000017
:104770003C840000D20400101E000010E80F00105E
:10478000C40400107013001064860000281000108C
:10479000F8B54F464646C0B40D1C40239946202329
:1047A00098461027461C047863B2002B05DA0020D7
:1047B00011210122FDF7F8FC04E000201121002264
:1047C000FDF7F2FC00200E210122FDF7EDFC002098
:1047D0000E210022FDF7E8FC4B46234205D00020C5
:1047E00011210122FDF7E0FC04E00020112100224C
:1047F000FDF7DAFC00200E210122FDF7D5FC002098
:104800000E210022FDF7D0FC4346234205D00020B4
:1048100011210122FDF7C8FC04E000201121002233
:10482000FDF7C2FC00200E210122FDF7BDFC002097
:104830000E210022FDF7B8FC274205D000201121EF
:104840000122FDF7B1FC04E0002011210022FDF758
:10485000ABFC00200E210122FDF7A6FC00200E215A
:104860000022FDF7A1FC230705D50020112101221C
:10487000FDF79AFC04E0002011210022FDF794FCD2
:1048800000200E210122FDF78FFC00200E210022C6
:10489000FDF78AFC630705D5002011210122FDF7F1
:1048A00083FC04E0002011210022FDF77DFC0020A4
:1048B0000E210122FDF778FC00200E210022FDF7D9
:1048C00073FCA30705D5002011210122FDF76CFC24
:1048D00004E0002011210022FDF766FC00200E21DB
:1048E0000122FDF761FC00200E210022FDF75CFC97
:1048F000E30705D5002011210122FDF755FC04E056
:10490000002011210022FDF74FFC00200E21012282
:10491000FDF74AFC00200E210022FDF745FC013D79
:10492000301C002D00D03DE70CBC90469946F8BDE8
:1049300070B5051C0C1C002011210122FDF734FC70
:1049400000E01D1C00201021FDF766FC061C701EF7
:10495000864100200E210122FDF726FC00200E21B9
:104960000022FDF721FC7600F6B200201021FDF7B1
:1049700053FC002801D00136F6B200200E2101229E
:10498000FDF712FC00200E210022FDF70DFC760041
:1049900000201021FDF740FC002801D00136F6B2BE
:1049A00000200E210122FDF7FFFB00200E21002236
:1049B000FDF7FAFB7600F6B200201021FDF72CFC83
:1049C000002801D00136F6B200200E210122FDF7A9
:1049D000EBFB00200E210022FDF7E6FB7600F6B28D
:1049E00000201021FDF718FC002801D00136F6B296
:1049F00000200E210122FDF7D7FB00200E2100220E
:104A0000FDF7D2FB7600F6B200201021FDF704FC82
:104A1000002801D00136F6B200200E210122FDF758
:104A2000C3FB00200E210022FDF7BEFB7600F6B28C
:104A300000201021FDF7F0FB002801D00136F6B26E
:104A400000200E210122FDF7AFFB00200E210022E5
:104A5000FDF7AAFB7600F6B200201021FDF7DCFB83
:104A6000002801D00136F6B200200E210122FDF708
:104A70009BFB00200E210022FDF796FB6B1C2E7085
:104A8000013C002C00D05CE770BDC04600B583B08F
:104A900000200F210122FDF787FB68460730012126
:104AA000FFF746FF03B000BD30B583B00B4C6D4639
:104AB00007350BE0281C0121FFF73AFF2B78FF2B6D
:104AC00006D00020642101F0DBFC013C002CF1D178
:104AD000631E9C41E0B203B030BDC04688130000A5
:104AE00010B582B000200F210022FDF75DFB684663
:104AF00007300121FFF71CFFFFF7D6FF041E02D18C
:104B0000FFF7C4FF00E00124201C02B010BDC04626
:104B100030B583B0041C0D1C43B2002B08DA7F2390
:104B20001C4037200021FFF7F3FF031C012B35D871
:104B3000FFF7ACFFFFF7D4FF031CFF20002B2DD0A5
:104B4000402323436A4613702B0E53702B0C937033
:104B50002B0AD37015719523002C00D00123082C4B
:104B600000D187236A46537168460621FFF710FE7D
:104B70000C2C04D1684607300121FFF7D9FE0A2426
:104B80006D460735281C0121FFF7D2FE287843B275
:104B9000002B03DA013CE4B2002CF3D103B030BDAA
:104BA00030B583B0051C0C1CFFF77EFF00281BD01E
:104BB00001A804700121FFF7EBFD0120FD2C13D0AB
:104BC000281C80218900FFF7E3FD01AC201C022195
:104BD000FFF7AEFE201C0121FFF7AAFE23781F205D
:104BE000184005384342584103B030BDF0B583B09A
:104BF000071C0E1CFA24A40001AD0BE0281C0121A7
:104C0000FFF796FE2B78FF2B06D10020642101F0E0
:104C100037FC013C002CF1D101AB1A780020FE2AB0
:104C200008D1381C311CFFF783FE01A80221FFF7D1
:104C30007FFE012003B0F0BD08B500201B21FDF769
:104C4000EBFA0138431E9841C0B208BD08B50020F8
:104C50001B210022FDF768FA08BDC04630B583B0BD
:104C6000124B1D78032400281AD11B21FDF7D4FA1A
:104C7000012815D006232C1C9C43EB0710D43A20A6
:104C80000021FFF745FF002801D001231C4301A8A4
:104C90000421FFF74DFE00200F210122FDF784FAC9
:104CA000024B1C70201C03B030BDC0462300001016
:104CB000F0B583B0FFF7D2FF051CAA0700D587E047
:104CC00000200F210122FDF76FFA0A2405E001A858
:104CD0000121FFF72DFE013CE4B2002CF7D10020AA
:104CE0000021FFF715FF0026012862D10820D521F9
:104CF0004900FFF70DFF012833D101AC201C04212E
:104D0000FFF716FEA378012B53D101ABDB78AA2B5A
:104D10000CD04EE0A920311CFFF7FAFE00280CD081
:104D20000020391C01F0ACFB013C04E0FA24A40093
:104D30008026F605271C002CECD10026002C38D04C
:104D40003A20311CFFF7E4FEB04232D101AC201C06
:104D50000421FFF7EDFD237804265A0629D50C26F9
:104D600027E0A9200021FFF7D3FE012383429B41C6
:104D70005B420226F61AFA24A400271C0AE0A920A6
:104D80000021FFF7C5FE002806D00020391C01F0E5
:104D900077FB013C002CF2D1002C09D0102080219F
:104DA0008900FFF7B5FE434243415B421E4000E0ED
:104DB0000026084B1E70002E02D0FE20054002E0A7
:104DC00001200543EDB2044B1D70FFF75FFE281C68
:104DD00003B0F0BDE90400102300001070B50D1CF5
:104DE000161C1C1CFFF73AFF0323C20737D4042309
:104DF000002C34D01B4B1B781A0700D47602012CF0
:104E00000FD11120311CFFF783FE002822D1281C6E
:104E100080218900FFF7EAFE434243415B421C4088
:104E200018E01220311CFFF773FE002812D18026F3
:104E3000B600281C311CFFF7D9FE002806D08023BD
:104E40009B00ED18013CE4B2002CF2D10C200021B3
:104E5000FFF75EFEFFF71AFE631E9C41E3B2181CCB
:104E600070BDC046E9040010F8B50E1C171C1D1CCF
:104E7000FFF7F4FE0324C20741D4022443073ED4C3
:104E80000424002D3BD01F4B1B781A0700D47F024F
:104E9000012D0ED11820391CFFF73AFE002829D128
:104EA000301CFE21FFF77CFE434243415B421D4024
:104EB00020E006221A4203D09720291CFFF728FE83
:104EC0001920391CFFF724FE002813D1301CFC21C7
:104ED000FFF766FE002806D080239B00F618013DF0
:104EE000EDB2002DF2D10020FD21FFF759FE002880
:104EF00000D10125FFF7CAFD6C1EA541ECB2201CB4
:104F0000F8BDC046E904001070B584B00C1C151C37
:104F1000FFF7A4FE031C0320D90750D4012C0DD0A9
:104F2000002C02D0032C42D045E0FFF7D9FD01242C
:104F3000002841D0FFF7AAFD00243DE00920002110
:104F4000FFF7E6FD0124002836D168461021FFF75F
:104F50004DFE002830D06A4613789B09012B0AD1F8
:104F6000527A6E46337A1B02D31801339BB29B02EE
:104F70002B60002420E05079937ADB09527A0F21CC
:104F80000140591803231A40520089186A46147ABE
:104F9000D2796E46B079A4099200A21803409B0210
:104FA000D2180132CB1F9A402A60002404E08023EB
:104FB0002B60002400E00424FFF768FD201C04B0EF
:104FC00070BDC04630B583B01D48FDF779FF0120A4
:104FD000FBF7AEFB0128FAD01A4B5878996A01F01A
:104FE0001FFE6D4607350120FBF7A2FB041C0020C5
:104FF00001F0E2FE002808D0002001F0E3FE287056
:105000000120291C012201F0BBFE012001F0D4FE89
:10501000002808D0012001F0D5FE28700020291CAE
:10502000012201F0ADFE002CDDD00748FDF748FF5E
:10503000044B5878596801F0F3FD03B030BDC04609
:105040005C8B0000E80F0010688B0000F0B557463D
:105050004E464546E0B488B0041C0F1C85783D3DA3
:105060006B425D41002D04D00330804601F08EFF7D
:105070008146667823781B023343C54CA34200D196
:1050800099E300D984E0C34A934201D100F0D2FCF5
:105090003ED8C14A934200D113E11CD8BF4A934283
:1050A00000D189E209D8BE4A934200D140E1BD4A0D
:1050B000934200D1AAE200F010FDBB4A934200D116
:1050C00004E2BA4A934200D139E3B94A934201D08B
:1050D00000F003FD62E2B74A934200D129E309D808
:1050E000B54A934200D108E3B44A934200D1E8E2C2
:1050F00000F0F3FCB24A934200D1E7E0B14A934298
:1051000000D1E8E0B04A934201D000F0E6FCC9E0EB
:10511000AE4A934200D137E21CD8AD4A934200D147
:1051200015E209D8AB4A934200D1E5E1AA4A93427D
:1051300000D1F4E100F0D1FCA84A934200D116E27C
:10514000A74A934200D10AE3A64A934201D000F055
:10515000C4FCF8E2A44A934200D1CAE009D8A34AA9
:10516000934200D124E3A24A934200D117E300F016
:10517000B4FCA04A934200D18AE39F4A934200D1F3
:10518000AEE39E4A934201D000F0A7FC00F059FC28
:105190009B4A934200D1D7E040D89A4A934200D12B
:1051A000CAE01ED8984A934201D100F068FC09D8A1
:1051B000964A934200D173E2954A934200D181E12D
:1051C00000F08BFC934A934200D171E1924A9342E2
:1051D00000D137E2914A934201D000F07EFC00F00A
:1051E00062FC8F4A934200D102E209D88D4A934271
:1051F00000D119E28C4A934200D165E200F06DFCC7
:105200008A4A934200D1E5E1894A934200D1B2E053
:10521000884A934201D000F060FC61E2864A9342E2
:1052200000D1C9E31DD8854A934200D1F2E309D8E1
:10523000834A934200D183E0824A934200D187E0BF
:1052400000F04BFC804A934200D119E27F4A93421E
:1052500001D100F0FDFB7E4A934201D000F03DFCFD
:10526000FEE17C4A934200D1B6E30DD87A4A9342DC
:1052700000D178E3794A934200D184E3784A93429B
:1052800001D000F02AFC48E3764A934200D1B3E310
:10529000754A934200D158E3744A934201D000F01A
:1052A0001CFC6BE0002D02D0714B49461970704B0D
:1052B00018780021002201F095FE01F01BFF00F09C
:1052C0000CFC6C48FEF7E4F900F007FC6948FEF7B7
:1052D000FFF900F002FC002D02D0674B4A461A701D
:1052E000654B18780021002201F07CFE01F002FFDE
:1052F000F3E303A9614A0B1C31CA31C312CA12C3BA
:1053000000245F4E5B4D5F4F0FE0A20003ABD2580D
:105310003260281CFEF70AFA306800F08FFD386012
:10532000281CFEF7F3F90134A4B2042CEDD9D4E320
:105330005048FEF7EBF9D0E34E48FEF7F7F9CCE31F
:105340004C48FEF71DFAC8E34A48FEF735FAC4E3B5
:105350004D4D4E4B2B60474C201CFEF711FA172386
:105360005B422B60201CFEF70BFA494B2B60201C84
:10537000FEF706FAB1E3FEF731F9AEE3002D00D1F6
:105380008AE04D46012D00D084E0FEF7BFFA83E0AD
:1053900057490000544400004443000053410000BA
:1053A0004C410000504100005242000043430000C5
:1053B0005A410000574300004F4300005243000091
:1053C00044440000494400004244000056470000A5
:1053D0004C4700004247000046470000534700008A
:1053E0005447000050470000414800005847000063
:1053F0005A47000052490000544900004D4800003F
:105400004554000052500000524D0000534C000023
:10541000434D0000584D000041500000574D000022
:105420004153000054500000435200005453000008
:10543000565300004C530000415A00005A540000DB
:1054400049540000545400005455000043580000D3
:1054500041550000505A00004D5A00004F5A0000BC
:10546000435A0000535A0000545A0000525A000098
:10547000780D001050890000B8040010488B00001F
:10548000C41700106013001094150010B5F7FFFF4B
:1054900094110000FEF7C2FAD24B1B68002B03D117
:1054A000D14801F095FD18E3D04801F091FD14E3D7
:1054B000CF4B18680021002201F094FDCD4801F087
:1054C00087FD0AE3CC4ACA4B1A6006E3002D02D0DE
:1054D000CA4B48465860C94B58680021002201F069
:1054E00081FD01F007FE002D00D1F6E2C34B587894
:1054F000596801F095FBF0E2002D02D0BF4B494600
:105500009962BE4B986A0021002201F06BFD01F008
:10551000F1FD002D00D1E0E2FDF7A4F8DDE2002D61
:1055200003D02D23B54A4C46D4542D23B34AD05C26
:105530000021002201F056FD01F0DCFD002D00D11C
:10554000CBE22D23AD4AD05CFCF7F4FFC5E2002D81
:1055500003D02C23A94A4D46D5542C23A74AD05C0E
:105560000021002201F03EFD01F0C4FDB5E2A34D93
:105570002424285DFA1E414601F002FC285D9D4965
:10558000022201F0FDFBA8E29D4801F021FDFDF79C
:10559000B3F801F01DFD01F0ADFD9EE2002D02D03B
:1055A000964B48461872954B187A0021002201F05C
:1055B00019FD01F09FFD90E2002D02D08F4B49466E
:1055C00059728E4B587A0021002201F00BFD01F038
:1055D00091FD82E2002D02D0884B4A46DA60874B6B
:1055E000D8680021002201F0FDFC01F083FD74E287
:1055F000002D02D0814B4C461C61804B1869002164
:10560000002201F0EFFC01F075FD66E2002D02D0F2
:105610007A4B4D461D75794B187D0021002201F013
:10562000E1FC01F067FD58E2002D02D0734B4846C3
:105630009861724B98690021002201F0D3FC01F0BF
:1056400059FD4AE2002D02D06C4B4946D9616B4BA3
:10565000D8690021002201F0C5FC01F04BFD3CE2BD
:10566000002D03D02023654A4C46D4542023634A9E
:10567000D05C0021002201F0B5FC01F03BFD2CE2E2
:10568000002D03D021235D4A4D46D55421235B4A8A
:10569000D05C0021002201F0A5FC01F02BFD1CE2F2
:1056A000002D02D0554B48465884544B588C00214D
:1056B000002201F097FC0122524B1A8001F01AFDE2
:1056C0000BE2FBF74BF808E2002D00D105E249465A
:1056D000012902D1FDF7AEFEFFE1FDF72FFFFCE14E
:1056E000002D00D1F9E14A46012A02D1464B1A7039
:1056F000F3E10022444B1A70EFE1444B1B78002B7E
:1057000000D0EAE1FFF798FA002800D1E5E103A80C
:1057100010213F4AFDF72AFD3E4803A90A22FBF764
:105720006FFF021E00D1D8E13B483C4901F004FF65
:10573000D3E138483A494246FCF78EFBCDE1354883
:10574000FCF74AFAC9E1002D02D0364B4C461C70DA
:10575000344B18780021002201F044FCBDE14046A2
:1057600001F0DAFB142102F0B1FB041C2E48604367
:105770002E4902F0ABFB850028188500281C2B4918
:1057800002F0A4FB061C281C284902F09FFB009194
:1057900021482749221C331C01F0CEFE9DE14046E2
:1057A00001F0BAFB021C1C48224901F0C5FE94E13D
:1057B000FFF708FC91E1404601F07CFC824644463C
:1057C000023400253BE0002B38D06378002B35D025
:1057D0006E1C201C01F06EFCAD00174968500234AD
:1057E000351C2CE06C0D0010748B0000788B0000D1
:1057F000C01700105089000019FCFFFFE80F0010CF
:105800007C8B00001E000010D3040010D204001096
:105810002C840000C817001079770000948B0000DA
:1058200064860000A4040010F42C0000102700007F
:10583000B88B0000C88B00001005001001342378DD
:10584000002BC0D1A84801F0C3FB504601F00EFC6C
:10585000A64801F0BDFBEAB29146101C01F006FC1F
:1058600001F048FC0024A24FA24E07E03B5DD8B2F5
:1058700001F0FCFB301C01F0ABFB0134AC42F5DB6A
:1058800001F038FC50469C494A46FDF731F924E1C5
:10589000404601F00FFC051C4046023001222A431D
:1058A000D2B2934B1A7001F005FC041C8E4801F033
:1058B0008FFB281C01F0DAFB8C4801F089FB201CCF
:1058C00001F0D4FB01F016FC8B4E281C311C221C6D
:1058D000FDF756F9301C211C002201F013FCFCE0FE
:1058E000404601F0E7FB071C4046023001F0E2FBB6
:1058F00003AE30704046043001F0DCFB041C7E4DEA
:105900000090381C311C01222B1CFDF767F9281C64
:10591000211C002201F0F6FBDFE0002D03D02E2336
:10592000764A4C46D4542E23744AD05C002100227F
:1059300001F058FB01F0DEFB002D00D1CDE02E235D
:105940006E4AD05CFAF708FEC7E0002D02D06B4B20
:105950004D461D63694B186B0021002201F042FB8C
:1059600001F0C8FBB9E0002D03D02F23634A48465D
:10597000D0542F23614AD05C0021002201F032FB79
:1059800001F0B8FBA9E02E235C4AD35C002B00D0C9
:10599000A3E0002D05D04946CAB201200121FCF741
:1059A00003FC01200121FCF737FC0021002201F05B
:1059B00019FB01F09FFB90E0002D03D03C234F4AE0
:1059C0004C46D4543C234D4AD05C0021002201F0C7
:1059D00009FB01F08FFB80E0002D03D03423474A00
:1059E0004D46D5543423454AD05C0021002201F0B5
:1059F000F9FA01F07FFB70E0002D02D03F4B4846E2
:105A000098633E4B986B0021002201F0EBFA01F005
:105A100071FB62E0002D03D03D23384A4946D15442
:105A20003D23364AD0560021002201F0DBFA01F076
:105A300061FB52E0002D50D04A46D0B2FDF774FA17
:105A40004BE0FCF7A3FE2E4B18802E48FDF7D0FE4E
:105A5000002D0CD04B46002B02D0012B04D006E0C9
:105A6000002001F023FC02E0012001F01FFC484669
:105A70000021002201F0B6FA01F03CFB2DE0404687
:105A800001F0EEF9072828D9404601F0D1F9046861
:105A900001F006FB3A20FDF741FB201C01F000FB62
:105AA00001F028FB19E0404601F0DAF9102814D97A
:105AB000404601F0BDF9051C4046093001F0B8F937
:105AC000041C2860281C01F0EBFA3A20FDF726FBA5
:105AD000201C01F0E5FA01F00DFB08B01CBC90465B
:105AE0009946A246F0BDC046D08B0000D88B00007E
:105AF000EC0C00108C82000010050010E80F001064
:105B0000580D00105089000038B5002001F054F9FC
:105B1000002800D185E0002001F054F9414B1870B5
:105B2000031C613BDBB2192B02D820383D4B1870A7
:105B30003C4B1B78202B74D0DAB2202A04D8082BD7
:105B400033D00D2B24D055E02A2B4DD0512B41D0F2
:105B5000212B4FD13448FDF7B3F92120FDF7DEFAB0
:105B6000324A334B1A60334A334B1A600023324CAB
:105B70002F4808E02268511C216001684D1C056017
:105B8000097811700133C72BF4DDFDF76DF848E09B
:105B900001F0B0FA294C21782948FFF757FA22780A
:105BA000284B1A70002323703BE0244B1B78002BFA
:105BB00037D0013BDBB2214A13700021204AD15477
:105BC0000820FDF7ABFA2020FDF7A8FA0820FDF722
:105BD000A5FA26E0194B1B78002B22D1194B197816
:105BE0001748FFF733FA1CE0144B1B78002B01D148
:105BF000FDF76AF80B4B1878031C203B5F2B10D87D
:105C00000E4B1B78132B0CD8FDF788FA0B4A117832
:105C10004B1CDBB213700A4A024800785054002132
:105C2000D15438BD0C050010E08B0000C92C0000D9
:105C30000805001000080010EC0400100D0500100D
:105C4000F00400101009001008B51E2000211E22CB
:105C500000F0A6FB08BDC04608B540006038C0B2E1
:105C60001021002200F09CFB80B208BD38B5FFF780
:105C7000EBFF0024054D05E0201CFFF7EDFF63005E
:105C800058530134072CF7DD38BDC046001A001008
:105C900070B500240025002616E0442000211522BE
:105CA00000F07EFB00201821002200F079FB36185E
:105CB00054200021152200F073FB0020182100223F
:105CC00000F06EFB2D180134032CE6DDB608034B03
:105CD0001E60AD08024B1D6070BDC046181A001052
:105CE000141A0010094B5B891B02094A1268D31A67
:105CF000084A1360084A1268002A06D00121064AA1
:105D00001160D917054A136051607047001A0010DE
:105D1000141A0010F01900102C000010F8190010CF
:105D200010B50B4B1868C1170A4B9A89002302F073
:105D30000AF94C02C20D2243CB15044902488018CF
:105D4000594110BDC046C046D00700000000000009
:105D5000F0190010001A0010F8B55F4656464D467F
:105D60004446F0B42D4B1B78012B14D12C490A6802
:105D70002C4B1B68D3180B602B498B4202D80A208E
:105D80002849086029498B4203D90A214942254BF9
:105D90001960101C3BE0264B19688946254B1C688E
:105DA0005D68254B5A88924699888846DA889346DA
:105DB0001A89201C291C002302F0C5F88B068609CD
:105DC0001E438F114146CB0B4A04B6185F41201C7D
:105DD000291C5A46002302F0B6F84C06C209224399
:105DE000CB110024002551460C0412196B41484682
:105DF000002102F0A8F8CC02420D22434B15141CDE
:105E00001D1CA41BBD416A04E40B101C20433CBCB8
:105E100090469946A246AB46F8BDC046780D0010A4
:105E20003400001028000010E7030000C0D4010077
:105E3000181A0010F8190010001A001008B50E4BBF
:105E40001B78022B13D10D4A10680D4B1B68C31829
:105E500013600C4A934203DD39214942084A11601C
:105E6000094A934206DA3922054B1A6002E0002102
:105E700001F016FA08BDC046780D00103000001081
:105E800024000010289A010030F8FFFF08B5EC202C
:105E90001E21FCF755FE08BD10B582B041006039E7
:105EA000C9B2EC20FCF74CFE6C460634EC20211CF9
:105EB0000222FCF765FE201C022101F001F9208876
:105EC00002B010BDF8B5FFF7E1FF0024064E074F02
:105ED00006E06500AF53201CFFF7DEFFA853013436
:105EE000072CF6DDF8BDC046001A00100F27000091
:105EF000F0B5474680B482B000230193009300249C
:105F000000250026FA239B0098461F4F32E04046AA
:105F100000F09AFAEC204221FCF712FE381C00F047
:105F200093FAEC200021FCF70BFEEC2001A90322E0
:105F3000FCF726FE01A8032101F0C2F8019BF61828
:105F4000404600F081FAEC205221FCF7F9FD381CA4
:105F500000F07AFAEC200021FCF7F2FDEC20694613
:105F60000322FCF70DFE6846032101F0A9F8009B0F
:105F7000ED180134002CCADD044B1E60044B1D607B
:105F800002B004BC9046F0BDE2040000181A0010F4
:105F9000141A001010B5CF4B1B78DBB20A2B00D9B6
:105FA000BDE19B00CC4AD3589F46CC4B1B68022BCB
:105FB00011D0042B1DD0012B00D0B0E10122C74B22
:105FC0001A6001200521FCF7EFF8012005210022CD
:105FD000FCF7AAF8A3E10222C04B1A6001200521B8
:105FE000FCF71AF9002800D099E10122BC4B1A7085
:105FF00095E1BA4B04221A6002225A6000225A61CB
:106000000122B44B1A708AE1B44B1B68022B15D0E5
:10601000042B1CD0012B00D081E1B04A1360B14A9F
:106020001278B1490978D2B20A41134200D176E11F
:10603000012005210122FCF7B7F870E10222A74BED
:106040001A60012005210122FCF7AEF867E1042265
:10605000A24B1A60A44B1A780132D2B21A701B7884
:10606000082B24D10022A04B1A70A04B1A880132B1
:1060700092B21A801A889E4B1B8892B29A420DD116
:106080000322944B1A70012005210022FCF74CF8E2
:10609000924B02225A6000225A6140E1934B1B88C6
:1060A000944A1268D3181A78D2B28E4B1A708B4C5D
:1060B00002236360012005210122FCF735F801204D
:1060C00005210022FCF770F80123636027E1834B70
:1060D0001B68022B11D0042B24D0012B00D01EE111
:1060E00001227E4B1A6001200521FCF75DF801209A
:1060F00005210022FCF718F811E10222774B1A6003
:1061000001200521FCF788F8002800D107E1764B33
:106110001B78DBB201229A40724B19780A43D2B243
:106120001A70FCE004226D4B1A606F4B1A78013232
:10613000D2B21A701B78082B1FD16C4B1A886D498C
:1061400009688A1867490878C0B2107000220A707E
:1061500065490A701A88013292B21A801A88644B13
:106160001B8892B29A4208D105225A4B1A705B4B97
:1061700002225A6000225A61D1E0584C0223636027
:10618000012005210122FBF7CFFF0120052100227C
:10619000FCF70AF801236360C1E0504B1B68022B37
:1061A00011D0042B18D0012B00D0B8E001224B4BAA
:1061B0001A60514B1B78002B00D1B0E00120052163
:1061C000FBF7F2FFABE00222444B1A6001200521ED
:1061D0000122FBF7E9FFA2E0404C042323600722E1
:1061E0003C4B1A70012005210022FBF79DFF022382
:1061F00063600023636192E0384B1B68022B11D06F
:10620000042B1CD0012B00D089E00122334B1A60F3
:1062100001200521FBF7C8FF012005210022FBF723
:1062200083FF7CE002222D4B1A6001200521FBF741
:10623000F3FF002873D001222F4B1A706FE0274B19
:1062400004221A600921234A117002225A60002296
:106250005A6164E0214B1B68022B10D0042B2BD019
:10626000012B5CD101221D4B1A6001200521FBF797
:106270009BFF012005210022FBF756FF4FE0022281
:10628000164B1A6001200521FBF7C6FF002809D034
:106290001A4B1B78012B42D1184B1A780132D2B21B
:1062A0001A703CE0154B1B78002B38D1134B1A7831
:1062B0000132D2B21A7032E00422084B1A600F4B3E
:1062C0001B78022B1CD10B22024B1A700222034BAB
:1062D0005A6024E011090010EC8B000000400140DE
:1062E0001E0900101F0900102009001018090010D5
:1062F0001C09001014090010120900101A090010DE
:10630000074C02236360012005210122FBF70CFFEB
:10631000012005210022FBF747FF0123636010BD28
:1063200000400140064B0122DA6119681968013109
:106330005960044B1A70044B1A6801321A60704796
:10634000000005401C1A0010201A001008B500209B
:1063500016210122FBF7E8FE00200F210122FBF7A6
:10636000E3FE00200E210122FBF7DEFE00201021BB
:106370000022FBF7D9FE002011210122FBF7D4FEF9
:10638000002016210122FBF70FFF00200F21012220
:10639000FBF70AFF00200E210022FBF705FF08BDD6
:1063A000F8B5051C0E1C171C002016210022FBF757
:1063B000FBFE002417E0EA0900201121FBF7F4FEA0
:1063C0006D00EDB200200E210122FBF7EDFE00234F
:1063D00001E0C0460133092BFBDD00200E21002225
:1063E000FBF7E2FE0134072CE5DD0020112100223D
:1063F000FBF7DAFE0025002416E06D0000200E21D8
:106400000122FBF7D1FE002301E0C0460133092B36
:10641000FBDD00201021FBF7FFFE054300200E21CD
:106420000022FBF7C1FE0134A642E6DC002F03D0B8
:106430000020391C00F024F8002016210122FBF76F
:10644000B3FE281CF8BDC046002315E0C046C04678
:10645000C046C046C046C046C046C046C046C0460C
:10646000C046C046C046C046C046C046C046C046FC
:10647000C046C04601339BB28342E7D37047C04653
:1064800038B50D1C00281BD11C4C0223636000236F
:10649000E3601B4B996F1B4B186801F01AFD1A49FA
:1064A00001F017FD4543A561FF23236004236361C9
:1064B00001236360211C01224B681A42FCD11CE0BD
:1064C00001281AD1114C022363600023E3600C4BB6
:1064D000996F0C4B186801F0FCFC0B4901F0F9FCBA
:1064E0004543A561FF2323600423636101236360A7
:1064F000211C01224B681A42FCD138BD00800140AA
:1065000000800440880400101027000000C00140F3
:1065100038B50D1C002818D1194C022363600023E4
:10652000E360184B1868FA21890001F0D2FC45435A
:10653000A561FF2323600423636101236360211CA1
:1065400001224B681A42FCD119E0012817D10E4CE8
:10655000022363600023E3600A4B1868FA21890074
:1065600001F0B7FC4543A561FF2323600423636169
:1065700001236360211C01224B681A42FCD138BD03
:10658000008001408804001000C001402C4B1B68B3
:10659000DA0706D501222A4B1A602A4B1A68013203
:1065A0001A60274B1B689A0706D50222244B1A60F3
:1065B000244B5A6801325A60214B1B685A0706D592
:1065C00004221F4B1A601F4B9A6801329A601C4BC1
:1065D0001B681A0706D50822194B1A60194BDA688E
:1065E0000132DA60164B1B68DA0606D51022144B0E
:1065F0001A60154B1A6801321A60114B1B689A0613
:1066000006D520220E4B1A600F4B5A6801325A6091
:106610000B4B1B685A0606D54022094B1A600A4BE1
:106620009A6801329A60064B1B681A0606D58022CA
:10663000034B1A60044BDA680132DA607047C046D7
:106640000080014024090010340900102C4B1B6805
:10665000DA0706D501222A4B1A602A4B1A68013242
:106660001A60274B1B689A0706D50222244B1A6032
:10667000244B5A6801325A60214B1B685A0706D5D1
:1066800004221F4B1A601F4B9A6801329A601C4B00
:106690001B681A0706D50822194B1A60194BDA68CD
:1066A0000132DA60164B1B68DA0606D51022144B4D
:1066B0001A60154B1A6801321A60114B1B689A0652
:1066C00006D520220E4B1A600F4B5A6801325A60D1
:1066D0000B4B1B685A0606D54022094B1A600A4B21
:1066E0009A6801329A60064B1B681A0606D580220A
:1066F000034B1A60044BDA680132DA607047C04617
:1067000000C001404409001054090010002803D1C2
:106710000122034B5A6002E00122014B5A6070478C
:106720000080014010B500285FD100291BD1594BD2
:106730009A6C07218A439A64986C032210439864E8
:10674000D86C8843D864D86C1043D864586D88439B
:106750005865586D10435865986D88439865996DD4
:106760000A439A6594E001291CD14A4BB0201A587B
:1067700007218A431A501C58032214431C5098685E
:1067800088439860986810439860D8688843D860B8
:10679000D8681043D86018698843186119690A439A
:1067A0001A6175E002291FD13A4B802299580720BF
:1067B000814399509C5802210C439C5084229C5840
:1067C00084439C509C580C439C5088229C58844382
:1067D0009C509C580C439C508C229C5884439C5049
:1067E00098580143995053E0FEE700291BD1294BEB
:1067F0001A6E07218A431A66186E03221043186620
:10680000586E88435866586E10435866986E884391
:106810009866986E10439866D86E8843D866D96E8D
:106820000A43DA6634E001290FD11A4B9A6907212D
:106830008A439A619869032210439861D869884312
:10684000D861D9690A43DA6122E002291FD1114BCC
:10685000E02299580720814399509C5802210C430B
:106860009C50E4229C5884439C509C580C439C5060
:10687000E8229C5884439C509C580C439C50EC222A
:106880009C5884439C5098580143995000E0FEE77F
:1068900010BDC0460040044070B5141C002825D12E
:1068A000264B5D6840222A435A6080229E588025EC
:1068B000AD0035439D50FFF735FF0023204D0022EA
:1068C000204803E099004A510A500133032BF9D9BB
:1068D0001D4B9C61DC611C625C621C4A9A621C4A12
:1068E0005A61802212021B4B1A6025E0012823D135
:1068F000124B5D68802215435D609E588025ED0037
:1069000035439D50FFF70EFF0023134D0021134820
:1069100003E09A00515111500133032BF9D9104B68
:106920009C61DC611C625C62084A9A62084A5A6196
:1069300080225202074B1A6070BDC046008004409E
:106940002409001034090010008001406D0B000084
:10695000DB06000000E100E04409001054090010CB
:1069600000C0014043011B18DB00154AD318013356
:10697000FF335A799B79D2B29A420FD3104B42011E
:106980001118C90059180131FF3149791218D20084
:106990009B180133FF339B79C81A10E0084B420162
:1069A0001118C90059180131FF3149791218D20064
:1069B0009B180133FF339B79C81A0130FF307047B1
:1069C000241A001070B5041C0E1CFFF7CBFFFE2824
:1069D00012DC0A4B62011519ED005D190135FF3516
:1069E0006879C0B2411CC9B269711119C90008188F
:1069F000181846712B1C5B7970BDC046241A001014
:106A000038B5041CFFF7AEFF002818DD0D4B6201FE
:106A10001019C00018180130FF308179C9B24D1C1F
:106A2000EDB285711019C000411859184879C0B2EB
:106A30001419E4001B190133FF339B7900E0002097
:106A400038BDC046241A001008B51D4B9B681B07B3
:106A50005B0F032B14D11A4B5B69FF2213409E225C
:106A60001A4204D0174A1360154B1B6827E0DA0757
:106A700025D5134B1968C9B20020FFF7A3FF1EE00C
:106A8000022B06D10E4B1968C9B20020FFF79AFFFE
:106A900015E0062B06D10B4B1968802252000A43E1
:106AA0001A600CE0012B0AD1054B5B699A0603D5ED
:106AB0000122044B1A7102E00022024B1A7108BD38
:106AC00000800040241A001008B5214B9B681B076A
:106AD0005B0F032B16D11E4B5B69FF2213409E22D6
:106AE0001A4206D0842252001A498B50184B1B6858
:106AF0002DE0DA072BD5164B1968C9B20120FFF734
:106B000061FF24E0022B06D1114B1968C9B20120A4
:106B1000FFF758FF1BE0062B08D10E4A84235B00C9
:106B2000D058802149000143D15010E0012B0ED1F3
:106B3000074B5B699A0605D5012186235B00054A50
:106B4000D15404E0002186235B00024AD15408BDE1
:106B500000C00040241A001010B5002823D10029DD
:106B60000FD12E4B9A6C07218A439A64986C0222AB
:106B700010439864D86C8843D864D96C0A43DA64AB
:106B80004AE0012948D1254B5A6F07218A435A67A9
:106B9000586F042210435867986F88439867996F1D
:106BA0000A439A6738E0012835D100290FD11B4BE1
:106BB0009A6E07218A439A66986E0222104398665D
:106BC000D86E8843D866D96E0A43DA6624E0012974
:106BD00011D1124BEC2299580720814399509C58AF
:106BE00005210C439C50E8229C5884439C509858A3
:106BF0000143995010E0094BDA6A07218A43DA62AF
:106C0000D86A03221043D862186B88431863196B43
:106C10000A431A6300E0FEE710BDC046004004408E
:106C2000F8B50F1C43011B18DB004F4AD318012293
:106C30001A710133FF3300225A719A7100234A4EB0
:106C400045012D18ED00002403E0EA18B218547134
:106C50000133FF2BF9D9002842D180248022D202AF
:106C6000424B1A510021FFF777FF414B596804222C
:106C70000A435A601959802252010A431A51982234
:106C8000012199503B4C8321E16099583A4B186897
:106C900001F01FF90009391C01F01BF9030A6360B8
:106CA000FF23184020600323E3601023A36207231F
:106CB000A3606369211C60224B691340602BFBD1E8
:106CC00001E01A6801E02B4B01215A691142F8D109
:106CD0008022D202254B1A600522264B5A6041E0E1
:106CE000802480221203214B1A510021FFF734FF28
:106CF0001F4B596808220A435A6019598022920191
:106D00000A431A519C22012199501C4C8321E160B5
:106D10009958194B186801F0DCF80009391C01F08A
:106D2000D8F8030A6360FF23184020600323E36060
:106D30001023A3620723A3606369211C60224B69AF
:106D40001340602BFBD101E01A6801E00B4B0121DD
:106D50005A691142F8D180221203044B1A600522AD
:106D6000064B5A60F8BDC046241A001000E100E04E
:106D700000800440008000408804001000C00040F3
:106D800070B50B4E20230B4D0EE0002805D16C6929
:106D90002342FCD00C782C6004E074692342FCD0C0
:106DA0000C7834600131013A002AEED170BDC04642
:106DB00000C000400080004008B5FFF7D3FD431E2F
:106DC000984108BD10B5041CFFF7CCFD031C002042
:106DD000002B02D0201CFFF713FE10BD031C021C69
:106DE000303AD2B2101E09280DD91A1C613A052A70
:106DF00002D8573BD8B206E000201A1C413A052AB7
:106E000001D8373BD8B27047F8B5071C00230024DF
:106E10004E0006E01D01FFF7E1FF031C2B43013488
:106E2000E4B2B44202DA385D0028F3D1181CF8BD90
:106E300008B50421FFF7E8FF08BDC04603E0934210
:106E400009D1013001310378002B06D00A78002ADD
:106E5000F5D1002002E0012000E000207047C0468C
:106E6000021C002001E0013080B2135C002BFAD13B
:106E70007047C046F0B557464E464546E0B4051C3F
:106E80000F1C002808D1002903D13020FCF746F957
:106E90003BE030230B7038E00026002809DA002997
:106EA00003D12D20FCF73AF902E02D230B700126C7
:106EB0006D4201239946174C00239A461EE0A846CE
:106EC000281C211C01F005F8051E02D14B46002BA1
:106ED0000CD1281C3030C0B2002F03D1FCF71EF9B2
:106EE000D14603E0731CB855DEB2D1466543434634
:106EF0005D1B201C0A2100F0ECFF041C002CDED1DD
:106F0000002F02D0BE19002333701CBC9046994656
:106F1000A246F0BD00CA9A3B30B500E001300378CC
:106F2000002B05D01A1C303A092A01D92D2BF5D196
:106F300001252D2B01D101306D42002305E0990080
:106F4000CB185B00303AD31801300278111C30396D
:106F50000929F4D92E2A11D1013000220BE0990021
:106F6000CB1859000B1C0478002C03D0231C303B99
:106F7000CB1801300132032AF1DD01E0024A53430C
:106F8000281C584330BDC0461027000010B500E053
:106F900001300378002B05D01A1C303A092A01D998
:106FA0002D2BF5D12D3B5A4253415B420122134315
:106FB000002205E09400A218520030398A180130EE
:106FC00001780C1C303C092CF4D9181C504310BD1E
:106FD00010B5041C02E0FCF7A1F801342078002869
:106FE000F9D110BDF0B5474680B40D1C161E0C2E0D
:106FF00000D90C260023002E07D1291CFFF73AFFE9
:107000002FE0E1540133DBB201E0174C00210C2BDF
:10701000F7D91549FFF72EFF711E134ECBB29846D4
:10702000301CB446202709E0434603E05A1E845C26
:10703000C454D3B2002BF9D163461F70735C002B8C
:10704000F2D00023002D04D108E0EA540133DBB272
:1070500000E00549CA5C002AF7D102E00248FFF7C8
:10706000B7FF04BC9046F0BD6409001038B5051C9C
:107070000309054CE05CFCF751F80F231D40605DEF
:10708000FCF74CF838BDC0468C8C000010B5041CD1
:10709000000AFFF7EBFFE0B2FFF7E8FF10BDC046C4
:1070A00010B5041C000CFFF7F1FFA0B2FFF7EEFFD4
:1070B00010BDC04608B50121FFF7A6FEC0B208BD4D
:1070C000032908D004290BD0022911D10378427872
:1070D000027043700CE0037882780270837007E0DE
:1070E0000378C2780270C3704378827842708370EC
:1070F0007047C04608B50D20FCF710F80A20FCF7D1
:107100000DF808BDF0B55F4656464546E0B4061C8E
:107110000F1C9346002A03D02B48FFF759FF02E0CB
:107120002A48FFF755FF0022294B1A7400249A467B
:1071300098463DE021070ED1FFF7DCFF5B46002BB0
:1071400003D07019FFF7ACFF02E0A0B2FFF79EFF7B
:107150002048FFF73DFF75192878FFF787FF2020AB
:10716000FBF7DCFF2B781A1C203A5E2A08D8E217BE
:10717000120FA1180F2001408A1A41468B5408E0D3
:10718000E3171B0FE2180F210A40D31A2E22514693
:10719000CA54E3171B0FE2180F210A40D31A0F2B12
:1071A00005D10D48FFF714FF0948FFF711FF01341F
:1071B000251EBD42BED3FFF79DFFFFF79BFF1CBC02
:1071C00090469A46A346F0BD188C0000548C0000EF
:1071D000341C0010588400008C82000070B50E1C16
:1071E000151CFFF7F5FE002406E0305DFFF73EFFBB
:1071F0002020FBF793FF0134AC42F6D3FFF77AFF70
:1072000070BDC046031C00208B4203DBD80FD11792
:107210009A4248417047C046F8B54F464646C0B40A
:1072200081461C4B1B68834202DD1A4B58682CE0D8
:107230008923DB00174AD3580024834221DA164BF6
:10724000D05822E0E300DE59651CEB00DA59904685
:107250004846311CFFF7D6FF002810D04346991B43
:107260000C4BE4001C196468ED005B195868001BA6
:107270004A46961B704300F029FE201805E02C1C9E
:1072800000E0044F882CDDDD00200CBC90469946C0
:10729000F8BDC046380000104C0400007047C046DE
:1072A00008B5FFF7B9FFFFF7F9FF08BD30B51B4B75
:1072B00000221A628E2189005C582025AC435C5064
:1072C0001A62002301E0C0460133C72BFBD9134BE0
:1072D000186401225A64002159645A64191C4B6CC9
:1072E0001A42FCD00D4B41229A608E22920099588E
:1072F000802081439950191C0122CB681A42FCD08E
:10730000064B03221A6701225A67002159675A6700
:10731000191C4B6F1A42FCD030BDC046008004409F
:107320001F4B022210B51F491A601F4A2024D16743
:1073300000228E211A6289005858A04358501A62C0
:10734000C822C046013A002AFBD101211A645964BF
:107350005A645964596C124AC807FBD5412191609F
:107360008E21890050588024A0435050D8680121B4
:107370000B4A0842FAD0032010670020516750677B
:107380005167596F01221142FBD0054B9A67074A9A
:1073900000231360064A1360064A136010BDC046FE
:1073A000008004401F0001000480044094800440D9
:1073B000988004409C800440F0B5071C89B00D1CE7
:1073C000141C00262B78002B00D1B0E0252B00D018
:1073D000A8E06A786B1C002A00D1A8E0252A00D119
:1073E0009FE0002005902D2A02D10121AB1C0591C0
:1073F0001D1C2A786B1C302A05D1059A1D1C0223FE
:107400001A430592F5E70421101C88432A2802D16B
:107410000022101C08E0303A092AF9D9002216E0AF
:107420002E2908D1012001335D1E29782A29F7D1A0
:1074300022680434F7E730390491C9B2092906D823
:107440000028F0D10A256A4304995218EBE72B78FB
:107450006C3B59424B41ED182B78702B32D00CD835
:10746000632B4DD0642B15D0582B55D1211D049181
:1074700021680092059A019231E0752B35D0782B66
:1074800018D0732B48D12168231D049300293ED1C5
:1074900028493CE021680092059A201D6123049050
:1074A00001920293381C0A22012300F08EF836184C
:1074B000049C3AE00598231D2168049300920190F2
:1074C00061230DE03020B8477820B847231D04938E
:1074D0000598082321680093022303430193412365
:1074E0000293381C10220023DFE7211D049121683C
:1074F0000092059A612301920293381C0A22F2E756
:10750000231D0493236807A90B7000234B70381CBC
:10751000059B00F01DF8CAE72520B8472878B84732
:1075200003E01D1C2878B847013601354AE7301CB6
:1075300009B0F0BDA08C00000EB403B503AA08CAC0
:10754000191C0192FFF738FF02B008BC03B01847BE
:10755000F7B5141C00900191002A0FDD0A1C019957
:10756000501A1178002901D00132F8E7A04201DA5F
:10757000241A00E00C1C30259A0700D42025002690
:10758000D9070BD4261C002E04DDE8B2009A9047E0
:10759000013EF8E7E643F6172640A41B371C019985
:1075A0008B1BD85D002803D0009B98470137F6E776
:1075B000261C002E04DDE8B2009A9047013EF8E751
:1075C000E043C01704403819FEBDF0B587B0071C72
:1075D00000920C1E09D103AB30221A7059700C9A1C
:1075E000191C0D9BFFF7B4FF40E00022019293426B
:1075F00007D0009B0A2B04D1914202DA01224C42AF
:10760000019200226B466E46DA751636751C002C08
:1076100011D0201C009900F05CFC092902DD0E9BB2
:107620003A3BC91830313170201C009900F051FCF0
:10763000013E041CEAE7019B002B10D00C9A002AA3
:1076400009D00D9B9B0706D52D20B8470C9A012425
:10765000013A0C9203E0013D2D232B700024381CCD
:10766000291C0C9A0D9BFFF773FF201807B0F0BD83
:1076700008B50020011C021C00F008F8FCF7E0F936
:1076800008BD08B500F076FC08BD000070B5244CBC
:10769000A02200215200201C00F0B2F8C02000F00F
:1076A00083FA204D0021C022286000F0A9F8286844
:1076B0000023282218215A435943A21841180133A4
:1076C0005162082BF5D1221C1749002000F068F9FF
:1076D000802280235B01201C0021D20000F028F8CA
:1076E000261C124D2836291C321C012000F058F9A6
:1076F00080228023301C5B0150340021D20000F036
:1077000017F8291C221C022000F04AF9802280234D
:10771000201C0021D2005B0100F00AF870BDC046B9
:107720004C1C0010481C0010A78C0000A98C000005
:10773000F0B5C5680124AE071AD08026B600B24263
:107740000BD08026F600B24204D08026A640B2427A
:107750000ED102E0416A231C04E0064E5F1E0124A4
:10776000B74205D82A4301610160C361C2600024A9
:10777000201CF0BDFEFFFF00084908B50B6B013B64
:107780000B63002B05DB8B6A5A1C8A621870C0B22F
:1077900002E0283100F05AF808BDC0464C1C001029
:1077A00010B5021C1378002B01D00132FAE7CC5C33
:1077B000D4540133002CFAD110BD0000031C0B433C
:1077C00030B59A0711D1021C0B680B4C1D190B4CDC
:1077D0009D43254202D108C20431F5E7D9B21170A8
:1077E0000132002907D01B12F8E70023CA5CC254FB
:1077F0000133002AFAD130BDFFFEFEFE808080807A
:1078000008B500F0CDFB08BDC26820239A43436A47
:1078100010B5041CE2605B6882699A420DD000F0EA
:10782000F3F8E268074B134010221343626AE360E7
:107830005368A361236993602360E268024B13409D
:10784000E36010BDEFCFFFFFBFBFFFFFF8B5514AA8
:10785000CB68061C1A400C1CCA60980602D5081C8E
:10786000FFF7D2FFA268E368511C0EDA98050CD42A
:10787000022149428A1AA260902252021343E36015
:1078800023685A1C22601E7081E0434A1D1C1A4066
:10789000022A05D00022A26080221343E36054E054
:1078A0003E490B40802109028B420AD10021201C55
:1078B00000F0DCF9E168890602D5201CFFF7A4FF7F
:1078C000E56890235B02F0222B431201E36015422E
:1078D0001ED1606900F080FB00280BD06A0509D535
:1078E000636A236123600123E36192235B022B43DC
:1078F000E3600DE080277F01381C00F055F99423E8
:10790000E2685B022B431A4320612060E761E2607A
:1079100090210901226825690B4219D0636A996890
:107920008A4200D9111C491B09D1636A6A1C9A60FA
:107930002260E269511EA160DA602E7027E0281CE7
:10794000221C00F093F80028EFD0012040421FE0F5
:10795000511CF0B221601070626A276891688446F9
:107960008F4200D9391CE769491BD760580504D4F8
:1079700063460A2B01D0B94209DB00239560281C1D
:107980002560A360221C00F071F80028DDD1F0B260
:10799000F8BDC046FFFFF7FF8A10000010A00000EE
:1079A00070B50D1C061C101C141C00F00DF92B7872
:1079B000722B06D0772B07D0612B20D10823114AD8
:1079C00004E00023012201E004230222013529788A
:1079D0002B2905D0622908D104210A43012102E0A4
:1079E00003210A4302210B43F0E7E26066611A07B4
:1079F00006D5201C0021022200F038F900E0002406
:107A0000201C70BD0280000038B5436A041C056963
:107A100002689968C36813481840E06082201840E3
:107A2000022802D0012040421AE080204002184083
:107A300016D0914200D2111CA94209D1636AE268B2
:107A40009D60094B002013402560A060E36007E0C3
:107A5000491B281C221C00F009F80028EED0E1E7A1
:107A600038BDC046FFFFF7FFFFFFFEFFF7B5D56843
:107A700001900E1C141C5769EA0205D51023381C0E
:107A80001D4300F0A6FAA061114B1D4208D0381C1E
:107A9000A16900F0A7FA002813DB0E4B1D40E5603A
:107AA000321C381C019900F0A3FA801B431E984138
:107AB000404243005B08F61AA3699E19A66100289C
:107AC00005D0E268802313430120E3604042FEBDFD
:107AD00010000200EFFFFDFFF8B52E4FC51C3C68FB
:107AE000AD08002819D0002610E0216880228C46BD
:107AF000A368520591423ED11968626861450ED172
:107B000059689B68521803326260A360002CECD164
:107B10000C3000F081F9421C30D1002039E0AA423B
:107B200006DBE91C914203DB80239B05236020E0F8
:107B3000291C0A318A4210D980218905201C216024
:107B40000C30A90041186560A160521B80246405B7
:107B5000033A0C604A608B601BE0002B0BD1920053
:107B6000801A00F059F90130D7D080239B0523609B
:107B70006560201C0CE0261C1C1CC7E780239B05AD
:107B8000036045608460002E01D1386000E0B06081
:107B90000C30F8BD8C1D0010002803D080230C3859
:107BA0005B0503607047000010B5FFF795FF041EEA
:107BB00005D10449172200F01BFA00F006FA201C38
:107BC00010BDC046AB8C0000F0B5436AC56889B0F3
:107BD000041C476906690193AB0726D02B0716D40E
:107BE00000F02AF8381C00F0F1F92B0502D5301C02
:107BF000FFF7D2FF0F4BAD0DAD059D4207D103A896
:107C0000216A142200F0F1F903A800F0D1F8002154
:107C10001822606AFFF7F4FD201C00212822FFF7DC
:107C2000EFFD019B0020636201E00120404209B0AA
:107C3000F0BDC046000080AD38B5002803D000F08C
:107C40000BF9051C0EE0041C051C0748201800F069
:107C500003F9002801D001256D42A02328345B00E0
:107C60009C42F2D1281C38BD4C1C0010F7B53B4B90
:107C70000D1CC168041C161C47690091194269D08B
:107C8000381C00F0A9F90190002863D1012E04D01E
:107C9000022E07D0002E5DD123E0201C00F062F8F8
:107CA0002D181EE0381C00F094F9E168002804DA71
:107CB00080231943E16001264DE0626A26689368DB
:107CC0009E4200D9331CA6699B1926699B1B8E0610
:107CD00003D55268934200DA131C834200DA031C76
:107CE000ED18002D36DB009E636AB60404D52268C9
:107CF0009968914200D29A60A1698D420DDB20689B
:107D00009A68824200D2021C20695618361AB5427F
:107D100003DCDF68CE19B54207DB009E002120227C
:107D2000A160616032435D6010E0009E6D1AB6078D
:107D300001D5EF1BA760009EF60702D5821AAA188C
:107D40006260009A4519202325609A43044B1A402B
:107D5000E26001E0022601960198FEBD03001000DA
:107D6000BFCFF7FFC368990705D1104B212201202F
:107D70001A60404218E0202219030BD5134202D0AA
:107D8000436A586804E0036881695A180369D01A85
:107D9000013809E0134202D0436A586804E00368DE
:107DA00081695A180369D01A7047C04674090010D7
:107DB00010B5041C00F006F8011C201C00F00FF99F
:107DC00010BD000010B5411C820706D00130431ED3
:107DD0001B78002BF8D1401A18E003680C4A9C1855
:107DE0000C4A9C43144201D10430F6E7DCB2421C39
:107DF000002C0AD0FF242402821C234205D0FF2439
:107E00002404C21C234200D0021D501A10BDC046DB
:107E1000FFFEFEFE8080808070B50C4C2368002B36
:107E200001D10B4B2360C61C256803239E43AE196A
:107E3000301C00F035F8002802D12660281C04E030
:107E4000044B0C2201201A60404270BD901D0010AE
:107E5000941D001074090010C36870B5041C032041
:107E600018401AD09A0605D5636A201C5D68FFF792
:107E7000CBFC04E02368A2699D182369ED1AE2682F
:107E8000064B201C1340E360FFF7BEFD291C061CB7
:107E90000022201CFFF7EAFE301C70BDFFCFFFFF61
:107EA000084B6A469A4202D90123904207D2064BF8
:107EB000002B01D1002302E09842FBD30123181CC0
:107EC0007047C046941D00100000000003000B43E3
:107ED00021D4002931D00122D207030901E0090190
:107EE00012099942FBD9430801E04900520899421E
:107EF000FBD900E04908401A07D35241FAD30146A2
:107F00001046704749084018F7D29218FAD3401823
:107F1000014610467047CB0F00D04942021000D5F1
:107F20004042534008B5FFF7D4FF0CBC521000D3B9
:107F30004042002A00D549421847F446002000F08C
:107F400001F86047704710B543435143C918040C0A
:107F5000130C5C43091992B2040C544380B243439E
:107F600050432204240C801861411A041B0C801811
:107F7000594110BD8446830708D18B0706D1131FD2
:107F800004D304C904C0043BFBD21A1D524205D0DD
:107F9000891A801A8B5C83540132FBD1604670478A
:107FA0008446043A09D3830707D109060B0A19430B
:107FB0000B0C1943043A02C0FCD2043203D0017006
:107FC0000130013AFBD160467047FEE70120404294
:107FD0007047012040427047012040427047012015
:107FE00040427047012040427047012040427047A4
:107FF000101C7047D01F0000AA1F0000BC1F00000B
:10800000C41F0000C41F0000C41F0000C41F0000E4
:10801000C41F0000C41F0000C41F0000C41F0000D4
:10802000C41F0000C41F0000D41F0000C41F0000B4
:10803000C41F0000C41F0000261F0000C41F000052
:10804000BC1F0000C41F0000C41F0000C01F0000B0
:10805000222A2B2C3A3B3C3D3E3F5B5D7C7F00005F
:10806000EBFE904D53444F53352E30004E4F204E73
:10807000414D45202020204641543332202020000D
:108080004E4F204E414D4520202020464154202077
:1080900020202000726D632E446174653A202564AF
:1080A0000D0A000024206E6F7420666F756E642EBA
:1080B00020626164206D6573736167652E0D0A002F
:1080C0004D65737361676520636865636B73756D78
:1080D000205B253032585D20213D2063616C637543
:1080E0006C6174656420636865636B73756D205B98
:1080F000253032585D2E0D0A00000000504D544BC3
:108100000000000047474100524D43002C20000072
:10811000556E6B6E6F776E0024504D544B36303574
:108120002A33310D0A000000436F6D6D20457272D5
:108130006F7200002628000090290000902900009E
:10814000902900009029000090290000902900004B
:10815000902900004A280000902900009029000082
:10816000902900009029000090290000902900002B
:10817000902900007028000090290000902900003C
:10818000902900009029000090290000902900000B
:10819000902900008029000090290000902900000B
:1081A00090290000902900009029000090290000EB
:1081B000902900009C2800009029000090290000D0
:1081C00090290000902900009029000090290000CB
:1081D000902900009C2800009029000090290000B0
:1081E00090290000902900009029000090290000AB
:1081F000902900009029000090290000902900009B
:10820000902900009029000090290000902900008A
:1082100090290000F4280000902900009029000017
:10822000902900009029000090290000902900006A
:10823000902900008029000090290000902900006A
:10824000902900009029000090290000902900004A
:1082500090290000182900009029000090290000B2
:10826000902900009029000090290000902900002A
:10827000902900005C2900006977623A2000000024
:1082800069773A20000000006972623A200000001D
:1082900069723A2000000000697772623A2000009B
:1082A000BC3000004A2F00008E2F0000AC2F0000D1
:1082B0000E3000006E3000000000010002000400DB
:1082C00008001000200040008000000100020004AF
:1082D00000080010002000400080030006000C0091
:1082E00018003000210000030006000C00180030C8
:1082F0004020C0008001FF3F00000011220049041F
:108300006D15E42E892A0001000A8020C03F401527
:1083100000204004004000223F2206005B044F047E
:1083200066046D047D0407007F046F0409000A00E1
:10833000000A4104802003147F1577040F153900CB
:108340000F11790471043D04760409111E00700AAE
:108350003800B602B6083F0073043F08730C6D0482
:1083600001113E0030223628802A62144926390045
:1083700080080F0023000800800058087C0458047F
:108380005E04582001150C0C740400101021001B11
:108390000011541454045C04031561090014080C02
:1083A00040151C0004081C10402C80124820400A74
:1083B0000011802452040828000102030201050470
:1083C0000405060707060300010101000000010182
:1083D00000000000010101004E3F0000643F00006A
:1083E0007A3F0000B83F0000E43F00002840000052
:1083F0005840000086400000C0400000FC400000E3
:1084000024410000504100004572726F72206D6F70
:10841000756E74696E672064726976652E0D0A0048
:10842000434647205265616400000000303A73748F
:1084300061727475702E74787400000025730D0AD3
:10844000000000005554433A20253034642D253077
:1084500032642D2530326420202000002530326423
:108460003A253032643A2530326400007A372D6C78
:108470006F672E74787400004572726F72206F708F
:10848000656E696E67206C6F672066696C65206633
:108490006F722077726974653A2025640D0A0000B6
:1084A0003D3D3D3D3D3D3D3D3D3D3D3D3D3D3D3DFC
:1084B0003D3D3D3D3D3D3D3D3D3D3D3D3D3D3D3DEC
:1084C0003D3D3D3D3D3D3D3D3D3D3D3D3D3D3D3DDC
:1084D0003D3D3D3D3D3D0D0A000000005A37204125
:1084E0006C74696D65746572204D6F64756C650D93
:1084F0000A00000028632920323031352C204865DD
:1085000078706572742053797374656D730D0A0DFC
:108510000A00000056657273696F6E3A20322E327F
:10852000340D0A004275696C6420446174653A2018
:108530004F637420313320323031360D0A00000091
:108540004861726477617265205265762025630DFB
:108550000A0D0A00203A20537461727475700D0A76
:1085600000000000303A6C6F67253034642E63736E
:1085700076000000303A4C4F47253034642E637348
:1085800076000000303A475053253034642E74781A
:10859000740000004572726F72206F70656E696EB4
:1085A0006720646174612066696C6520666F722063
:1085B00077726974653A2025640D0A00203A204FCD
:1085C00070656E656420646174612066696C652005
:1085D000257320666F722077726974650D0A00003A
:1085E000203A204F70656E6564206770732066695D
:1085F0006C6520257320666F722077726974650D33
:108600000A000000203A20436C6F736564206461A7
:1086100074612066696C650D0A000000203A2043F1
:108620006C6F736564206770732066696C650D0AF2
:1086300000000000303A74657374312E7478740051
:108640004572726F72206F70656E696E6720666921
:108650006C6520666F7220726561643A2025640A39
:108660000000000025730A00303A6C6F673030302C
:10867000302E7478740000004572726F72206F7033
:10868000656E696E672066696C6520666F7220771B
:10869000726974653A2025640A0000004F6E6520F7
:1086A000627269676874206D6F726E696E672C20E4
:1086B000696E20746865206D6964646C65206F66FE
:1086C00020746865206E696768742C0A00000000D9
:1086D00074776F206465616420626F797320676FBF
:1086E0007420757020746F2066696768742E20206E
:1086F0004261636B20746F206261636B0A0000004B
:1087000074686579206661636564206561636820CB
:108710006F746865722C206472657720746865696F
:10872000722073776F7264732C20616E640A00008C
:1087300073686F742065616368206F746865722E5A
:10874000202041206465616620706F6C6963656DEF
:10875000616E20686561726420746865206E6F695F
:1087600073652C0A00000000616E642063616D6512
:1087700020616E64206B696C6C6564207468652090
:1087800074776F206465616420626F79732E0A0AC2
:10879000000000004E6F7720696620796F752064B5
:1087A0006F6E27742062656C6965766520746865F4
:1087B0007365206C696573206172652074727565DC
:1087C0002C0A000061736B2074686520626C696E0E
:1087D00064206D616E2E20204865207361772069CA
:1087E0007420746F6F2E0A002863292032303135CF
:1087F0002C20486578706572742053797374656DA8
:10880000730D0A00253032643A253032643A25303F
:1088100032640D0A00000000475053204669726D13
:10882000776172652056657273696F6E203A2025F4
:10883000730D0A0D0A00000043256C753D256C750B
:108840002025730044313D256C7525730000000020
:1088500044323D256C7525730000000044543D25CD
:10886000642573005A3D256425730000503D256C36
:10887000752E0000256C75257300000025642E25DB
:1088800030326400545F696E743D257325730000B7
:1088900025642E2564000000545F6578743D2573BF
:1088A00025730000484D3D256C642E0054696D65AC
:1088B0002C2050726573737572652C20545F496E5D
:1088C000742025632C20545F4578742025632C2068
:1088D000416C7469747564652025632C2056696E3B
:1088E0002C204144302C204144312C204144320082
:1088F0002C205554432C204C61742C204E2F532C8B
:10890000204C6F6E2C20452F572C205370656564CA
:108910002025732C2048656164696E672C204750C0
:108920005320416C7469747564652025632C20564E
:10893000616C6964000000002C2048756D696469F1
:108940007479202500000000496E69742049324383
:108950000D0A0000496E6974204C43440D0A000062
:108960005A4C4F47205A37580000000056455220B5
:10897000322E32340000000041444320496E6974B5
:1089800000000000544D5020496E69740000000042
:10899000505A5320496E6974000000004653204924
:1089A0006E69740043464720496E697400000000F8
:1089B00047505320496E6974000000004C4F472017
:1089C000496E697400000000436F6E736F6C650040
:1089D000202020475053204669726D7761726520D0
:1089E00056657273696F6E203A2025730D0A000078
:1089F00052756E6E696E67005A202536640000005D
:108A00004D202536640000002573202573000000EA
:108A100050202534642E2530326400002530326425
:108A200068253032646D25303264000056202025E0
:108A300032642E2530336400484D202532642E25C3
:108A400030326425250000002534642E253264254B
:108A5000630000002535642E253164256300000085
:108A600053202533642E253264000000482025332E
:108A7000642E253264000000475A25366400000049
:108A800025642C2025642E253032642C2025732C5F
:108A90002025732C2025642C2025642E253033645A
:108AA0002C2025642E253033642C2025642E25307F
:108AB00033642C2025642E253033642C2025642C2F
:108AC0002025642E253034642C2025632C20256439
:108AD0002E253034642C2025632C2025642E25304F
:108AE00034642C2025642E253034642C2025642CFD
:108AF0002025642C2025642E2530326400000000DF
:108B000025642C2025642E253032642C2025732CDE
:108B10002025732C2025642C2025642E25303364D9
:108B20002C2025642E253033642C2025642E2530FE
:108B300033642C2025642E253033642C2025642EAC
:108B400025303264000000005CD40100031C0000EA
:108B50007119000051110000E80300004750532034
:108B600042524447000000002020202020202020E6
:108B700000000000300D0A00310D0A00475053205C
:108B80004669726D776172652056657273696F6EA2
:108B9000203D20004572726F72206F70656E696EA5
:108BA000672066696C6520666F72207772697465EC
:108BB0003A2025640D0A000025642C2025642E250A
:108BC0003034640D0A00000025640D0A0000000026
:108BD000416464723D0000002043743D00000000C9
:108BE000535755504441544500000000AA5F00000F
:108BF0001E630000086000001E630000CE600000DD
:108C00001E6300009A6100001E630000F86100000E
:108C10001E6300005462000020202020202020201D
:108C200020202030202031202032202033202034EA
:108C300020203520203620203720203820203920C1
:108C40002041202042202043202044202045202075
:108C5000460D0A0020202020202030202031202016
:108C60003220203320203420203520203620203789
:108C7000202038202039202041202042202043205D
:108C800020442020452020460D0A00003031323398
:108C900034353637383941424344454600000000F8
:108CA000286E756C6C2900720077002A2A2A205FD2
:108CB000437379735F616C6C6F63206661696C6587
:048CC000640A00FF43
:108CC400F11FFF1F010001000B0000006D70680020
:108CD400006B706800000000000102000900010040
:108CE400DE07010139000000F6FFFFFF010000006C
:108CF40030F8FFFFC0D401006801000048E801001B
:108D0400BE010000C0D401002B02000038C10100E4
:108D1400B4020000B0AD010064030000289A010011
:108D240042040000A08601005C05000018730100E5
:108D3400C2060000905F010088080000084C010092
:108D4400C90A000080380100AA0D0000F8240100BF
:108D540056110000701101002F120000880D01004F
:108D640013130000A009010003140000B80501005A
:108D7400FF140000D001010007160000E8FD000008
:108D84001D17000000FA00004118000018F600004A
:108D94007219000030F20000B31A000048EE00001F
:108DA400041C000060EA0000651D000078E6000075
:108DB400D71E000090E200005C200000A8DE000046
:108DC400F4210000C0DA0000A0230000D8D600007F
:108DD40061250000F0D200003827000008CF000011
:108DE4002629000020CB00002D2B000038C70000EE
:108DF4004D2D000050C30000882F000068BF000004
:108E0400DF31000080BB00005434000098B700003C
:108E1400E7360000B0B300009B390000C8AF000083
:108E2400713C0000E0AB00006B3F0000F8A70000BD
:108E34008B42000010A40000D145000028A00000CF
:108E440041490000409C0000DD4C0000589800009F
:108E5400A6500000709400009E540000889000000A
:108E6400C9580000A08C00005F5B0000488A000025
:108E7400225D0000B88800005F5F0000C486000027
:108E8400A7610000D0840000FA630000DC820000C7
:108E940058660000E8800000C2680000F47E00000C
:108EA400386B0000007D0000BA6D00000C7B0000F0
:108EB4004870000018790000E27200002477000076
:108EC40089750000307500003C7800003C73000098
:108ED400FD7A000048710000CA7D0000546F000054
:108EE400A4800000606D00008C8300006C6B0000A7
:108EF400818600007869000084890000846700008E
:108F0400948C000090650000B38F00009C63000007
:108F1400E0920000A86100001C960000B45F00000D
:108F240067990000C05D0000C09C0000CC5B00009D
:108F340028A00000D8590000A0A30000E4570000B6
:108F440027A70000F0550000BEAA0000FC53000053
:108F540065AE0000085200001CB20000145000006E
:108F6400E3B50000204E0000BBB900002C4C00000B
:108F7400A3BD0000384A00009DC100004448000021
:108F8400A7C5000050460000C4C900005C440000AE
:108F9400F1CD00006842000031D2000074400000AE
:108FA40083D60000803E0000E7DA00008C3C00001D
:108FB4005EDF0000983A0000E7E30000A4380000F8
:108FC40083E80000B036000033ED0000BC3400003C
:108FD400F6F10000C8320000CDF60000D4300000E5
:108FE400B8FB0000E02E0000B8000100EC2C0000EB
:108FF400CB050100F82A0000F40A0100042900004E
:109004003110010010270000841501001C25000008
:10901400EC1A0100282300006A200100342100001A
:10902400FE250100401F0000A82B01004C1D00007C
:1090340069310100581B0000413701006419000028
:109044002F3D010070170000354301007C1500001E
:109054005349010088130000884F01009411000057
:10906400D6550100A00F000062580100D80E000080
:10907400F35A0100100E0000875D0100480D000046
:109084001F600100800C0000BB620100B80B0000EF
:109094005B650100F00A000000680100280A000076
:1090A400A86A010060090000546D010098080000DE
:1090B40004700100D0070000B97201000807000025
:1090C40072750100400600002E780100780500004A
:1090D400EF7A0100B0040000B47D0100E803000051
:1090E4007D800100200300004B8301005802000032
:1090F4001C86010090010000EE880100C8000000F9
:10910400CD8B010000000000A28E010038FFFFFF9C
:109114008691010070FEFFFF74940100A8FDFFFF1B
:1091240058970100E0FCFFFF509A010018FCFFFF74
:109134003E9D010050FBFFFF36A0010088FAFFFFAF
:1091440038A30100C0F9FFFF00366E0100366E013E
:0400000300000115E3
:00000001FF
